:020000020000FC
:0200000037C007
:02000800567828
:100034000C94512B0C944F2B4156522D43686970EC
:100044004261736963322028632920323030362DAF
:1000540032303038204A6F65726720576F6C667291
:04006400616D0000CA
:10007000F894A0E02A2EA1E03A2EA0E1AEBFAFEFA7
:10008000ADBFB0E0A0E0AA95F1F7BA95D9F70E940C
:10009000E12C0E9419390E940E790E94B1340E940D
:1000A0003B2EAFEFA093310120923D0120923E0103
:1000B000209250018827789420922D01A091290147
:1000C000A4FD0C946A000E943B2E0E9489010E94AC
:1000D0009732CECFA1E00E94B12DAA270E945B2DBE
:1000E0009927A7E10E94AC2D0E943B2EA0E10E941F
:1000F000AC2DC4E0DAE0E7E3F7E10E947F31A7E04E
:100100000E94AC2D0E9430300704200071D1A6E17E
:100110000E94AC2DC5E0D8E0E6E0F9E00E947F3116
:10012000D8E1F9E10E947F31D8E0F9E0CC5FEC5FE3
:10013000C833A0F366E90E946E326A95E1F70C9429
:10014000A100A0E00E94B12DA1E00E9423349927D4
:1001500020922A01AA270E945B2DA5E10E94AC2DC6
:100160000E943B2EC0E0D0E0EDE1F4E10E94D331EB
:10017000A1E50E94AC2D0E94303001084156522D5D
:100180004368697042617369633200003BD24091F9
:100190003D014B3008F0442740933D01642F67FD3B
:1001A00066276B3008F06AE050E06F9334D16F91AE
:1001B00053955830D1F7FCD1D1D1A6D16F93A5D2A8
:1001C0006F91423E11F46A95EACF433E11F4639574
:1001D000E6CF443E21F4643010F06450E0CF453E59
:1001E00021F4673010F46C5FDACF6830F8F04A3EE3
:1001F00011F0443F19F760933D01683039F44A3EED
:10020000E9F604D10E94A31B01D19BCF693039F4D8
:100210004A3EA1F6FBD00E946D20F8D092CFF6D0D6
:100220004A3E61F60E943522F1D08BCF4F93409128
:10023000140142FD33C04F914A3E11F0443F41F456
:1002400060933D01E3D088270E948901DFD079CFF8
:10025000413F89F460933D010E941C7A3C96459190
:10026000423419F04F3F09F0A9CFD0D088270E941F
:100270007301CCD066CF423F39F460933D01C6D0C4
:100280000E94511DC3D05DCF433F39F460933D01BF
:10029000BDD00E94B61DBAD054CF90CF4F91413FF0
:1002A00039F460933D01B2D00E949B03AFD049CF97
:1002B000423F39F460933D01A9D00E94C922A6D0E3
:1002C00040CF433F39F460933D01A0D00E94042306
:1002D0009DD037CF443F09F760933D0197D00E94EE
:1002E000E30394D02ECFA0911601A030E1F70E9435
:1002F000570420922D01A0911701A43F09F021CFAE
:1003000008D00E949E32A0E00E945B2D0E943B2EEE
:10031000EACF0E943B2E8827209216010E941C7A69
:100320003C9645914E3411F4339609940E94F60D93
:1003300020920D012092500120922A010E94752ED8
:10034000A7E20E94AC2D92E0A0913E01A03079F08E
:10035000A33021F4A7E20E94AC2D09C0A0E10E94C5
:10036000AC2DA0E4A0930001A0EEA0930101A09108
:100370003E01A03051F40E9430301600205052450A
:1003800053532045534320002EC0A13051F40E9406
:1003900030306900205052455353204553432000CC
:1003A00022C0A23051F40E94303042002050524509
:1003B000535320455343200016C0A33049F40E94F4
:1003C00030302F00205052455353204553432000D6
:1003D000A53049F40E943030380020505245535324
:1003E000204553432000A0911601AD3EE1F708954A
:1003F0000E943030FF4156522D436869704261734C
:100400006963322056302E3837000895A0911601C6
:10041000A030E1F70895A1E0B3E050FDA95F51FDE0
:10042000A25F52FDBA5F4EE2651709F44295409310
:100430002C010E9449300E943030FF20200040E50E
:100440000E94A22E452F4F5C0E94A22E0E943030A7
:10045000FF202000B3950E944930452F0E941E7A4C
:100460003C9645914E3481F40E943030FF2020E6C6
:10047000E7202000B3950E9449300E943030FF20D1
:1004800020E8E920200021C0423481F40E9430306D
:10049000FF2020D0D1202000B3950E9449300E9437
:1004A0003030FF2020D2D32020000FC00E943030F7
:1004B000FF2020CACB202000B3950E9449300E9423
:1004C0003030FF2020CCCD202000452F0E941E7A06
:1004D000B3950E94493066E045910E94A22E6A952C
:1004E000D9F7B3950E94493066E045910E94A22E4B
:1004F0006A95D9F7B3950E9449300E943030FF20A9
:1005000020202020200008954AE26A3009F4429514
:1005100040932C010E9430300F0F202020202020FB
:1005200000000E943030100F2020D4D52020000081
:100530000E943030110F2020D6D7202000000E94CA
:100540003030120F20494E464F2000000E943030BC
:10055000130F2020202020200000089548E2693059
:1005600009F4429540932C010E9430300F0820205E
:100570002020202000000E94303010082020D8D9F0
:10058000202000000E94303011082020DADB2020DB
:1005900000000E9430301208434F4E464947000089
:1005A0000E943030130820202020202000000895D1
:1005B0004CE2683009F4429540932C010E9430309F
:1005C0000F0120202020202000000E943030100148
:1005D0002020DCDD202000000E943030110120208E
:1005E000DEDF202000000E943030120144464C41E2
:1005F000534800000E94303013012020202020208A
:1006000000000895A0E00E94AC2D0E94303015003B
:1006100020202020202020202020202020202020DA
:10062000202020202020202020202020202000000A
:10063000A7E20E94AC2D0E9430301600202020201E
:1006400020200000A0E60E94AC2D0E94303016064B
:100650002045646974200000A0E40E94AC2D0E9433
:100660003030160C2053617665200000A7E10E940F
:10067000AC2D0E9430301612204C6F6164200000B7
:10068000AEE6A0932B07A7E30E94AC2D0E9430306A
:1006900016182052756E20000895A0E00E94AC2D1F
:1006A000A7E20E94AC2D0E943030160020202020AE
:1006B00020200000A0E60E94AC2D0E9430301606DB
:1006C00020436F7079200000A0E40E94AC2D0E94AE
:1006D0003030160C2053656E64200000A7E10E94A4
:1006E000AC2D0E9430301612205265637620000037
:1006F000AEE6A0932B07A7E30E94AC2D0E943030FA
:100700001618436C6561720008953DED2092170143
:100710000E943B33409114014470431739F0342F49
:10072000403011F46FDFF4CFB8DFF2CF4091170102
:10073000403071F30895A4E00E94AC2DC1E0DFE0E9
:10074000ECE1F3E10E94D331A0E40E94AC2D0E94C1
:1007500030301002436F70792050726F6772616D94
:1007600020746F0070913D0160E0ACE0671709F400
:10077000A0E60E94AC2DB2E1A62FAA0FA60FAD5F96
:100780000E94493040E50E94A22E462F47704F5CE0
:100790000E94A22E6395683041F70E949732423E34
:1007A00021F47030D1F37A95DFCF433E21F47730D6
:1007B000A1F37395D9CF4A3E19F40E94517A089556
:1007C0004D3E59F708950E940E374F436C65617294
:1007D00020746869732050726F6772616D3F2000EA
:1007E000413009F008950E942B7A0895AA270E94AB
:1007F000B12DA3E00E9423348F9340913D010E94CC
:1008000024790E943B2E0E94502D99274091160179
:100810004030E1F70E94303000002050524F4752E4
:10082000414D200040913D014F5C0E94A22E4AE3C1
:100830000E94A22EC3EDD1E059D2F1D20E94EB79F1
:1008400004D48F91A8E8803069F1ACECE4E8F0E1E1
:10085000813031F0ABE48A9545914030E9F7F8CF2B
:100860004DD292E0A5E0B1E00E9449300E942830CC
:100870000E943030FF20494E2050000040913A0144
:100880004F5C0E94A22E4AE30E94A22EBB27AC2DF1
:10089000A3950E94CB2D4AE30E94A22EAD2DA395D5
:1008A0000E94CB2D0895AAE25A2E70E2089599274E
:1008B000FADF9CDFD22CAA27BB27D0922E010E9400
:1008C000C1320E943B33403E11F4AA27F6CF413E8D
:1008D00011F4AFE12BC0423E11F4AA9527C0433E6C
:1008E00069F4A3959B2F0E947B099A1730F4BE35BB
:1008F00011F4AA951BC0AA27B39518C0443E21F451
:10090000BA95B7FDBB2712C0463E21F4B850B7FDDB
:10091000BB270CC0473E11F4B85F08C0453E11F438
:10092000B39504C04A3E39F5B395AA27A03838F0EC
:10093000AFE1BA95B038C0F0AA27BB27BECFA0322E
:1009400028F0BE3589F0AA27B395B7CFBF3508F098
:10095000BEE50B2F0D1508F4D02E0D2D015F0B17E2
:1009600018F40B2F0F50D02E9B2F0E947B099A1743
:1009700008F4A92FA2CF9B2F4E3E39F4AF93BF931B
:100980000E943D09BF91AF918AC14F3E39F4AF93A8
:10099000BF930E944809BF91AF9181C1493E11F4B4
:1009A00082D17DC14C3E31F4A03009F488CFAA95A4
:1009B0007AD175C150911401547009F4C5C0433FF8
:1009C000D1F4ACEC9BD10E94303001075245434535
:1009D0004956452050524F4752414D20592F4E20E5
:1009E0003F006DD12EF48DD230D35DDF5092C8011F
:1009F0007DD1882760CF423F39F5ACEC7FD10E9492
:100A00003030010753454E442050524F4752414D1C
:100A100020592F4E203F000052D156F7ACEC6ED13A
:100A20000E943030010753454E44494E472E2E2E2A
:100A30002020202020202020000030922A0193D165
:100A400020922A0130DFD4CF443FB1F4ACEC56D130
:100A50000E9430300107434C4541522050524F47CD
:100A600052414D20592F4E203F0029D126F4DBD290
:100A70001ADF5092C801BCCF413F41F5ACEC3ED1EA
:100A80000E94303001075052494E542050524F4777
:100A900052414D20592F4E203F0011D1B6F4ABE406
:100AA0002DD10E94303001075052494E54494E47D3
:100AB0002E2E2E202020202020202000A2E0A093F7
:100AC0002A0151D120922A01EEDE92CF433671F4F1
:100AD00062E46093E50165E56093E60166E4609396
:100AE000E7016DE36093E80179D2E9CE483791F4EC
:100AF00062E46093E50165E56093E60166E4609376
:100B0000E7016DE36093E8010E94EE077CD250920A
:100B1000C80118C04637B1F46091E501623499F418
:100B200060E26093E5016093E6016093E701609302
:100B3000E8016093E9016093EA0143D286D25092C2
:100B4000C801BDCE8827BBCE423F11F5BF93AF93FE
:100B5000C9D0D9F0ACECD2D00E943030010753415B
:100B600056452050524F4752414D20592F4E203F5D
:100B70000000A5D046F40E94B7790E94EB7965D2B7
:100B800092DE7093C801B2D08827AF91BF9195CE05
:100B9000433FE1F4BF93AF93A5D0B9F0ACECAED036
:100BA0000E94303001074C4F5354204348414E4778
:100BB000455320592F4E203F000081D026F70E9438
:100BC000EB7943D270DE7093C801DDCF413F49F429
:100BD0006A2E7B2EADD0A62DB72D5092C8016FCEB8
:100BE000D2CF4D3E09F5BF93AF937CD0A9F0ACECCA
:100BF00085D00E94303001075155495420572F4F5E
:100C0000205341564520592F4E203F0058D046F7DB
:100C1000A0911601A030E1F70E94482DA0E00E94AB
:100C20005B2DAF91BF910895443FE1F45BD029F46F
:100C30000E94482D0E943B2E0895A9E65FD00E9495
:100C40003030010753415645204348414E474553F4
:100C5000204245464F52452052554E2100000E94E9
:100C6000973291CF5091140152FD1CC053FD1AC010
:100C70004C31C0F04038B0F4AF3171F05A2FAFE1D1
:100C80000E9416336A916983AA95A517D9F74883FC
:100C9000A3955092C80113CE0E94163348835092F8
:100CA000C8010DCE0CCE0E9416335A2F5F3121F0B1
:100CB000498149935395FACF50E2588308950E9491
:100CC0009732493559F0493749F04A3E39F04E34A8
:100CD00039F04E3629F04D3E19F0F1CF6894089561
:100CE000E8940895A091C801A0320895A8E806D01C
:100CF0000E94303001054F4B00000895EF93FF93A1
:100D00009927A09340010E94303001052020202027
:100D100020202020202020202020202020202020D3
:100D200020202020202020202000FF91EF910895F6
:100D3000A0E00E94E9324A3E09F40895423E21F4BF
:100D4000A030B9F3AA95F5CF433E21F4AB3089F337
:100D5000A395EFCF403268F3403858F74883AB3063
:100D600009F0A395E6CFC9ECD1E056E149910E9484
:100D7000A22E5A95D9F70E94752E4EE511D016F085
:100D80004A95E1F7542F53954427451719F024D07D
:100D90004395FBCF43E20E94A22E0E94752E089538
:100DA000CF93DF935F936F93E894C4E3D2E053E271
:100DB000459FC00DD11D50E26991613238F45A95BA
:100DC000D9F76F915F91DF91CF91089568946F91FA
:100DD0005F91DF91CF910895DF93CF934F935F930E
:100DE0006F93C1E3D2E053E2459FC00DD11DDF9365
:100DF000CF93A39653E26A91613210F45A95D9F7D2
:100E0000CF91DF9149910E94A22E5A95D9F70E9465
:100E1000752E6F915F914F91CF91DF910895AF93B0
:100E2000BF93EF93FF934F93AEE0B2E0E6E4FEE0B2
:100E30004591403011F04D93FBCF4F91FF91EF91D1
:100E4000BF91AF91089520457869742020204E61AC
:100E50006D6520202053617665202052656C6F619E
:100E60006420202052756E202000AF93BF93EF9333
:100E7000FF934F93AEE0B2E0E2E9FEE045914030EF
:100E800011F04D93FBCF4F91FF91EF91BF91AF9137
:100E9000089520202020202020205072696E742088
:100EA0002053656E64202020526563762020202028
:100EB0004E6577202000AF93BF93EF93FF934F933E
:100EC000AEE0B2E0EEEDFEE04591403011F04D9322
:100ED000FBCF4F91FF91EF91BF91AF9108952041CA
:100EE000626F7274202020202020202020202020CB
:100EF00020202020202020202020202020202020F2
:100F00002000D9DFACECFADE0E94303001055245FA
:100F100043454956494E472E2E2E000020922E0161
:100F20000E9413089927ECECE0934001E3EDF1E017
:100F3000EE2EFF2E41E10E942B345CE00E944734EC
:100F40004B31B9F14A33D1F70E9447344B3189F123
:100F5000403218F041935A95B9F7403228F00E9478
:100F600047344B3131F1F9CFEEE0F2E0EE2EFF2EB7
:100F700053E2EE2DFF2DB396EE2EFF2E0E94473446
:100F80004B31B9F04032D0F3433299F006C00E94A1
:100F900047344B3171F0403248F041935A95B9F7DC
:100FA0000E9447344B3129F04032D0F79395903668
:100FB000F9F60895A3E2BA9FA1E3B2E0A00DB11D36
:100FC0000895BF93AF93F6DFC8E7D1E053E24991AC
:100FD0004D935A95E1F7AF91BF910895BF93AF93A9
:100FE000E9DFC8E7D1E053E24D9149935A95E1F723
:100FF000409178014093E901409179014093EA01E1
:10100000AF91BF910895BF93AF934F935F93D2DF9A
:10101000139640E250E24D935A95E9F75F914F9154
:10102000AF91BF910895DF93CF93BF93AF934F9349
:1010300040E2A1E3B2E0CDEFDCE04D932197E9F788
:101040004F91AF91BF91CF91DF91DF93CF93BF933A
:10105000AF934F9341E0A1E3B2E0C0E3D42FDA5065
:1010600010F0C395FCCFD65CCD93DD93C0E2CD9359
:1010700090964395403689F74F91AF91BF91CF91AC
:10108000DF910895425245414B004F564552464C20
:101090004F5700444956494445202F300053515280
:1010A0002046524F4D203C3000434F4E5354414E4A
:1010B0005420544F4F204249470057524F4E47202B
:1010C00045585052455353494F4E0053594E544181
:1010D00058204552524F5200554E4B4E4F574E20BE
:1010E0004B4559574F52440057524F4E4720464F99
:1010F000524D415400424144204C494E454E554DBD
:10110000424552004E45585420572F4F20464F52CB
:101110000052455455524E20572F4F20474F53559C
:101120004200544F4F204D414E5920474F53554296
:1011300000544F4F204D414E5920464F52004932E6
:1011400043204552524F5200554E4B4E4F574E2062
:101150004552524F520044464C415348204552524A
:101160004F52004F5554204F462041525241590092
:10117000494E434F4D504C45544520504152004B31
:101180004559574F5244204953204D495353494ED6
:10119000470057524F4E472042434F505920004F6F
:1011A0005554204F462053435245454E0043414E2F
:1011B0004E4F54204352454154452046494C45002A
:1011C0004D454D4F52592046554C4C0046494C45D3
:1011D000204E4F5420464F554E4400504147452025
:1011E0004E4F5420494E2046494C450050414745FA
:1011F00053204E4F5420494E2052414E4745004EF9
:101200004F5420494E204752415048494353204DA6
:101210004F4445004E4F5420494E205445585420C9
:101220004D4F4445004E4F205553522046494C45A2
:1012300000535243204F5554204F462053435245AC
:10124000454E0044455354204F5554204F4620539B
:10125000435245454E0057524F4E47205350524936
:10126000544500494F2044495341424C4544004EA7
:101270004F204558544D454D0000BE3508F00895A7
:10128000BF9328D0B395BE35E1F7BDDEBF91DDCE6B
:10129000BE3508F00895BF93AF93AB2FAA95BDE577
:1012A00008D0BA95BA17E1F7B395ADDEAF91BF910B
:1012B000CCCEBF93AF93DF93CF937CDE1396ED013B
:1012C000B0E2A991AAA3BA95E1F7CF91DF91AF91CE
:1012D000BF910895BF93AF93DF93CF936BDE1396C7
:1012E000ED01B0E2ABA1A993BA95E1F7CF91DF91FF
:1012F000AF91BF910895BF93AF93DF93CF935ADE21
:10130000ED0193964E914132E8F34038D8F7AC1B8B
:10131000BC0B9A2F925097FD9927CF91DF91AF91F7
:10132000BF910895CAEEDCE02A922A9280E02F92C3
:10133000AA27BB27442771917032E9F37C3121F44D
:10134000A191BB27719156C07E3121F4A191BB2799
:10135000719150C07D3121F4B191A19171914AC038
:101360007F3121F4B191A191719144C07C3130F46D
:10137000572F4C2E5D2ECE2FDF2F63C07432C1F459
:101380007191703320F07A3310F4705305C07134CA
:1013900068F0773458F47753B03148F4A295B29599
:1013A0005A2F5F70A07FB52BA70FEACF23C029C0AB
:1013B000703350F17A3340F5403810F086E02AC19E
:1013C000AA0FBB1FF0F04A2E5B2EAA0FBB1FC8F05E
:1013D000AA0FBB1FB0F0A40DB51D98F07053A70F56
:1013E000B21D78F0B7FD0DC07191703318F07A33EB
:1013F00008F4E6CF4F3709F473D1AA93BA9340E8C3
:101400009DCF85E007C144C07134E8F37B35D8F740
:101410006081613458F16B3548F54C2E5D2ECE2F2E
:10142000DF2F21970C2F1D2FE0E9FBE152E0759192
:10143000703011F488E0EEC0703261F46991683266
:1014400099F45F93452FAA27BB27EC2FFD2FC42DBE
:10145000D52D71CF6991671751F375917032E9F706
:101460005395C02FD12FE3CF87E0D4C0403810F080
:1014700086E0D0C07154770FEF93FF93E0E9FCE072
:10148000E70FF21DA191B191FF91EF917191B2CF50
:101490007D3251F44F3711F444274DCF20F44032C0
:1014A00010F04FE748CF6FC0783231F471E07F938E
:1014B000AA27BB27472F3FCF793209F05EC05F9143
:1014C000513019F0523011F403D153C0533011F49C
:1014D00013D14FC0543029F4CCD1803009F09AC0D8
:1014E00046C0553029F4B991A991B095A0953FC057
:1014F000563009F4DDC1573009F48DC2583009F473
:101500009EC2593009F4B3C25A3009F4CAC25B30E2
:1015100009F4D2C25C3009F4D3C25D3009F4D5C2FB
:101520005E3009F4AFC2503109F40AC2513109F4F6
:1015300025C1523109F428C1533109F40EC2543186
:1015400009F423C25F3009F411C3553109F4BCC159
:10155000563109F4D0C1573109F4D5C1503029F0C2
:101560006ED0803009F056C0AACF86E00895AA93C5
:10157000BA93AA27BB2742E0DECE4F3720F44F3084
:1015800010F086E047C07C3361F471E260816E3315
:1015900019F472E2619142C06D3311F473E261910A
:1015A0003DC07E3339F474E260816D3311F475E22D
:1015B000619134C07D3311F476E230C07B3211F496
:1015C00070E32CC07D3211F471E328C0733211F442
:1015D00072E324C07A3211F470E420C07F3211F437
:1015E00071E41CC0753211F472E418C0763211F443
:1015F00073E414C05F91503021F05F3130F01FD0A0
:10160000F9CFB991A9913197089586E05F91503053
:10161000C1F3FCCF4F914030E9F708955F91A72FB8
:10162000B52FA07FB07FBA1720F009D0803091F796
:10163000F5CF5F937F93AA27BB27472F7CCE5F937D
:101640004F9319910991B991A991513211F4FED09A
:101650003AC0523221F4F3D0A150A17034C05332B9
:1016600021F4FCD0A150A1702EC0543211F4F6D058
:101670002AC0553221F4EAD0A150A17024C05632BC
:1016800011F4DDD020C0503311F441D01CC05133CF
:1016900011F43CD018C0523319F4A02BB12B13C055
:1016A000503411F43FD00FC0513411F4A7D00BC007
:1016B000523421F4A3D0A22FB32F05C0533419F410
:1016C000A023B12300C0AA93BA934F915F910895CC
:1016D000B991A99103D0AA93BA930895B7FF089539
:1016E000A095B095A30DB21D089517FF089500951C
:1016F0001095030D121D0895B991A991AB2B29F0F6
:10170000B7FBA1E0BB270EF41297E5CFF0DF2B2F3C
:101710002127A00FB11F27FD08952B2F212727FD7B
:1017200082E008950CD0A22FB32FBF770EF4D8DF3C
:1017300037FD03C0452B09F4089582E008957AD05F
:10174000CDDFB19F402D512DA09F202D312DA19F88
:10175000300D411D521DB09F300D411D521D089589
:1017600008E611E0B03818F0A00FB11FFBCFA017AA
:10177000B10718F0A01BB10BFACF0895B991A99148
:101780000AE5A01BB20902C0B991A991E9DFFF9354
:10179000EF93E0E6FAE70AE510E0A017B10748F496
:1017A000E00FF11FEA1BFB0BA491EF91FF91BB2708
:1017B000DECE04EB10E0A017B10778F40AE510E0E4
:1017C000E01BF10BEA0FFB1FA491EF91FF91BB27E8
:1017D000A095B095A30DB21DCACE0EE011E0A017E2
:1017E000B10728F4E00FF11FEA1BFB0BEDCF0EE071
:1017F00011E0E01BF10BEA0FFB1FD6CF212F202BAE
:1018000011F483E0089516D022273327442751E1AD
:10181000441FAA1FBB1F5A9551F0221F331F4FEFC1
:10182000201B310BA8F7200F311F40E0F1CF0EF441
:1018300057CF08952B2F212727FB50DF56CF0A279C
:101840001B27AA27BB27012B89F00895B0581058F1
:10185000A01BB10BAA27BB2748F00895B058105819
:101860000A1B1B0BAA27BB2708F00895A1E0B0E0D4
:101870000895B991A99184E0B7FD08950F931F933E
:101880002F933F9388270A2F1B2FB2E0AA27232DDF
:101890003327021B130B20F0A3952B0F321DF9CF1A
:1018A000BB27AA93BA933F912F911F910F9108954F
:1018B0004F935F930E94C0341991099142DFA42F86
:1018C000B52F5F914F9153CE19910991023039F4A0
:1018D00020925001A2E0A0933301BB2748CE0130F3
:1018E00031F4A0913301A03011F430923301A09172
:1018F0003301BB273CCE199109910EBD0E94F6170A
:10190000AEB5BB2734CE10913E01103011F08CE102
:10191000089519910991A4ECB2E00A171B0710F081
:1019200082E10895FF93EF93FDE0ECE3E00FF11FF8
:1019300068940E945E34EF91FF91A42FBB2717CECD
:10194000B991B0937301A991A0937201CF93DF93E2
:101950000E94FA17DF91CF910ACEB991A991BF3FAA
:1019600071F0A09358010E944D20803021F0AFEF1C
:10197000BFEF8827FCCDA42FBB270C94B70A0E9489
:1019800052208827B42FAA27F2CDB991A991BF3F41
:1019900021F5A0FD11C0DF93CF93FF93EF930E9439
:1019A0004A20803019F08827CC27DD27DE01EF910F
:1019B000FF91CF91DF91DBCDDF93CF93FF93EF9337
:1019C0000E944A20803019F08827EE27FF27DF0188
:1019D000EF91FF91CF91DF91CACDA09358010E9462
:1019E0004D20803021F08827AA27BB27C0CDDF9368
:1019F000CF937F9377270E945520DF3F41F4CF3F5D
:101A000031F4A72FBB277F91CF91DF91B0CD739594
:101A1000703889F7F6CFA991A991A770A06CA0930F
:101A20007C00A0917A00A064A0937A00A0917A0033
:101A3000A6FDFCCFA0917800B091790098CDB99126
:101A4000A991B03061F4AF3F79F0A770A395B0B120
:101A5000B695AA95E9F7AA27AA1FBB2788CDBA2F62
:101A6000A0B1AB23BB2783CDA0B1BB2780CDB9915B
:101A7000A9910E941A790E9460398030C9F4BB276D
:101A8000A52F75CDB991A991CF93DF93CA2FDB2FE5
:101A90000E949D39DF91CF91803051F4BB27A42F54
:101AA00066CDA99179910E947B39803009F45FCD90
:101AB000AA27BB278FE0AACDB991A991BB2757CD03
:101AC000B991A991AB2FBB2752CD0F93B991099131
:101AD000AA27BB27003019F4A091160145C0013098
:101AE00029F4A0911601A030E1F33EC0023039F490
:101AF000A0911601A030E1F7A091170135C0033085
:101B000019F4A091140130C0043039F4009114018B
:101B100000FD119602FD119727C0053039F40091A0
:101B2000140101FD119603FD11971EC0063049F402
:101B300000911601023E09F41197033EA9F4119693
:101B400013C0073049F400911601043E09F41196C0
:101B5000053E51F4119708C01F931091160101170B
:101B6000E1F71F91A02FBB270F9101CDB991A9914A
:101B7000BB27A13021F4A0916D01A395F8CCA23030
:101B800021F4A0916E01A395F2CCA0916F01EFCC4E
:101B90004142532053474E20535152204E4F542020
:101BA000524E442041444320494E20585045454B15
:101BB0002054454D50204C4F204849204B4559203A
:101BC000455045454B204552522041522053494EE5
:101BD00020434F53204654595045204653495A45B7
:101BE000205053544154205350492000FCE0E0E978
:101BF000A0E0B4EBA193BA95E9F7F1E0E8E6B0E133
:101C0000A193BA95E9F7FDE0ECE3B0E0A193A193CD
:101C1000A193BA95D9F7DD24CC2420920F0120920C
:101C20000D01AEE0A0932C01ACE3A0934401AEE221
:101C3000A0934501AFEFA09377010E943B2E209225
:101C40005001A2E0A0933301A6ECA0937A0040914A
:101C50003D0140933A01409337010E9424799C2D25
:101C60000E9440791FD0803039F4AC2DAF35B8F3E5
:101C70009CE0209250010895C0926D01D0926E01B7
:101C800080936F0120925001409177014F3520F4ED
:101C9000DD24C42E8827E3CF9CE0209250010895D4
:101CA000F70129C0F1E0E0EA20922A018827AD2D52
:101CB000BB27AB1701F171917F3FC1F17C31C9F0B6
:101CC0007E31B9F07D31A1F07F3191F0773271F141
:101CD000723241F471917F3F49F1773239F17232BA
:101CE000C9F7E9CF7A3339F7B395AB1721F703C0BA
:101CF00071917191E0CF70912D0170FF05C081E06D
:101D00007E7F70932D01089572FF0BC0AB7F70939F
:101D10002D01A0913E01A53011F0A03011F40E94D8
:101D20005A1B0E943B3371917F3F19F4DD24C39409
:101D3000089577FD2BC07032F1F27A3311F4D39409
:101D4000DACF773299F37134D8F07B3528F07052BE
:101D50007134B0F07B35A0F4672E0E9432177D33CA
:101D600079F4E0DA803069F4762D7154770FDCE095
:101D7000C0E9C70FD21DA993B99393CFEF91FF91FB
:101D800087E00895703810F487E08ACF7F01EDEC8A
:101D9000FEE07F73E70FF21D099445C0EDC0A0C2BD
:101DA00036C10CC1EDC22EC33EC736C337C33BC3D9
:101DB00034C08EC6ACC64CC3A2C3D4C2FAC32AC4B4
:101DC00078C16CC47CC481C4E9C195C286C491C485
:101DD00098C45AC54AC1D5C077C22BC1E2C49BC4BE
:101DE0001CC0E3C404C54EC2DDC2C5C5AAC717C620
:101DF00023C628C673C1AAC6F9C67BC729C638C67A
:101E00005AC215C55AC61FC181C297C300C393C425
:101E100099C43DC175C13CC692C188E0089584E172
:101E2000089583E108950E9436179CE0732C209258
:101E30002A01B191B032E9F3BA3311F0BF3F59F43E
:101E4000319770FC0E94752E40912A01443010F0A9
:101E50000E94203926CFBB3311F47724EACFBC325D
:101E600091F440912A01403031F40E94A12EBA2D04
:101E7000B770D9F706C00E94A12EB0912B01B770A0
:101E8000D1F77724D6CF732CB332C9F420925801FE
:101E90002092590147DA4A2F40932A01443018F41E
:101EA000433001F4C6CF0E942439683051F5509177
:101EB0002A015E7F0E942639683119F5BACFB03405
:101EC00011F5A0D740912A01433018F40E944930FF
:101ED000B0CF39F4A0935801B0935901A0932B01CE
:101EE000A8CF5FEF0E942639683259F45A2F0E941A
:101EF0002639683231F45B2F0E942639683209F4A2
:101F000098CF8FE00895B13229F40CDA9A2F91CF4F
:101F100097CF8FCFB23241F441914F3FC9F3423254
:101F2000C1F30E94A22EF8CFB63291F4FBD9B330A0
:101F300010F082E10895CCE3DDE0CA0FDB1F499188
:101F4000403029F00E94A22E1196B330C0F371CF19
:101F5000B53229F4E7D94A2F0E94A22E6ACF3197D1
:101F6000E1D9803009F00895903818F40E94CB2D03
:101F700060CF0E94262E5DCFA0E0F6D60E943B2EB9
:101F80008FCEA2E0F1D6A030C1F0A13059F0A091DF
:101F90005A01A770AA0FB0912C01B770A295BA2B65
:101FA000B0932C01A0915801A770AA0FB0912C01F9
:101FB000B07FBA2BB0932C0173CE33CFA3E0D4D62D
:101FC000A33018F1A0915801B0915901A09372016A
:101FD000B0937301A0915A01B0915B01A093580195
:101FE000B0935901A0915C01B0915D01B03011F442
:101FF000A03051F00D010E94FA170E948B17D001FA
:10200000803021F41197F2CF4BCE0BCF0895A5E08D
:10201000ABD6A43068F0B6D77F93E3D6E0936B01DC
:10202000F0936C010E945D317F9170932C0138CE4A
:10203000F8CEA1E099D6A130D8F340915801417073
:1020400040930D012DCEA5E08FD6A43068F09AD72D
:102050007F93C7D6E0936B01F0936C010E947F31B0
:102060007F9170932C011CCEDCCEA5E07DD6A430F0
:1020700068F088D77F93B5D6C0936B01D0936C017D
:102080000E945B367F9170932C010ACECACEA5E0E8
:102090006BD6A43068F076D77F93A3D6C0936B013C
:1020A000D0936C010E94AB367F9170932C01F8CDD8
:1020B000B8CEA3E059D6A23080F064D77F93B09118
:1020C0005801A0915A01A0936B01B0936C010E943A
:1020D0005C307F9170932C01E3CDA3CEA5E044D674
:1020E000A43068F04FD77F937CD6E0936B01F093D8
:1020F0006C010E9439327F9170932C01D1CD91CE29
:10210000A0913E01A03011F08CE10895A1E02CD601
:10211000A130A8F3A0915801B0915901CCE3DDE0C2
:10212000CA0FDB1F40912C014F93AF92BF920E94C8
:10213000F236BF90AF904F9140932C01B1CDA0915A
:102140003E01A03011F08CE1089575D6C093700166
:10215000D093710187D67C32F9F4A1E006D6A13084
:1021600070F2A0915801B0915901CCE3DDE0CA0FA3
:10217000DB1F40912C014F93AF92BF920E941B37FF
:10218000BF90AF90C0917001D09171014993299295
:102190004F9140932C0184CD87E082CDA0913E01E8
:1021A000A03011F08CE1089546D6C0937001D09311
:1021B000710158D67C3281F7A1E0D7D5A13009F062
:1021C00030CEFF93EF93AF92BF9240912C014F938B
:1021D0007F934F7040932C010E94BF19C1E0D2E061
:1021E000ECE1F5E10E94D331C0912C01C295C0937E
:1021F0002C010E94303003020000A0915801B091E0
:102200005901CCE3DDE0CA0FDB1FA6E14991403262
:1022100030F0403820F40E94A22EAA95B9F7772713
:1022200061E025D00E94E519623079F4C091700117
:10223000D0917101799329927F914F9140932C0114
:10224000BF90AF90EF91FF912BCD7F914F91409335
:102250002C01BF90AF90EF91FF91C0917001D09190
:1022600071014FEF499349931BCD87E019CD0E942F
:10227000D6178827603009F408950E94F51D882735
:1022800062E00895A3E070D5A230A0F07BD67F93E2
:10229000D0916C01C0916B01F0915801E0915A010D
:1022A000E0936B01F0936C010E9439327F9170933F
:1022B0002C01F6CCB6CDA4E057D5A43021F491D5AD
:1022C0000E943531EDCCADCDA1E04ED5A13090F0DE
:1022D000A0915801A295AA0FAF7EA0930F01E0CC68
:1022E000A1E042D5A13030F0A0915801A150CA2EF2
:1022F000DD24089596CDA1E037D5A130D8F3A09183
:102300005801A150A0937701CBCC8BCDA5E02CD563
:10231000A23030F1F1E0E0915801E770B0915A013C
:10232000B770BB0FB295B193A230C9F0E770B0910E
:102330005C01B770BB0FB295B193A33081F0E77029
:10234000B0915E01B770BB0FB295B193A43039F074
:10235000E770B0916001B770BB0FB295B193A0CC9C
:1023600060CD5FCDA1E000D5A130D8F3A091580198
:10237000A53009F0A3700E945B2D0E943B2E90CCEB
:10238000A1E0F2D4A13068F0A0915801B0915901B8
:10239000B03019F4A03009F483CC0E946E3211974A
:1023A000F7CF3FCD20925001A2E0A0933301A3E0EC
:1023B000DBD4A33020F1CCE3DDE0A0915801B09153
:1023C0005901B330E8F4AC0FBD1FA0935201A093A4
:1023D0005401B0935301B0935501A0915A01B091AB
:1023E0005B01B33068F4AC0FBD1FA0935601B093EE
:1023F0005701A0915C01A09350012092330150CC71
:1024000082E14ECC20925001BF91BF91089530D50A
:10241000AB2B09F48BCC45CC29D543CCF701F2D4B6
:102420000E9449303ECC24D50E9477323ACC672FA7
:102430006F931ED56F914A2F0E94A22E65FD0E94B8
:102440001F3311D57C3271F70DD50E949209F3CF5D
:10245000A2E08AD4A13019F0A23021F1E2CCA091FF
:102460005801AA95AF3510F08AE01ACCB0916F01EF
:10247000BF3010F08DE014CCAF93CCEEDCE0A5E0E3
:10248000AB9FC00DD11DB395B0936F01BD2DB3951A
:10249000B068B993BC2DB993B0913D01B993DD24D7
:1024A000CF900895A0915A01AA95AF35E8F6B09162
:1024B0005801BA95B770B0933701B0916F01BF3032
:1024C00010F08DE0EDCBAF93CCEEDCE0A5E0AB9F60
:1024D000C00DD11DB395B0936F01BD2DB395B068FC
:1024E000B993BC2DB993B0913A01B993DD24CF9043
:1024F0004091370140933A010E9424790895B6D45F
:10250000B0916F01B03011F48CE00895BA95CCEE23
:10251000DCE0A5E0AB9FC00DD11DB0936F01B99178
:10252000B7FFF2CFBF77DB2EC990499140933A01B4
:102530000E942479089587E0089598D493D4713443
:10254000D0F37B35C0F77154770F672E8BD47D3372
:1025500091F70E949209803009F00895DCE0C0E90B
:10256000C60DD21DA993B9937DD4743521F771910D
:102570007F3409F70E9492094A2E5B2E803009F0C1
:102580000895B0916F01BF3010F08EE00895CCEE49
:10259000DCE0A5E0AB9FC00DD11DB395B0936F01FA
:1025A000BD2DB395B993BC2DB993699249925992B7
:1025B00078CB5CD4B0916F01B03011F48BE008950A
:1025C000BA95CCEEDCE0A5E0AB9FC00DD11DB99172
:1025D000B7FDF4CFBF77B0936A0159907991BCE011
:1025E000A0E9A70FB21D0D911D91030D121D1E93A1
:1025F0000E93A991B99111960A1741F41B1731F462
:10260000B0916F01BA95B0936F014BCBC52CD090B0
:102610006A010895A0913E01A03011F08CE1089567
:1026200025D4BFEFB0937801B191B032E9F34B2FCD
:10263000BF3F21F40E94752E319733CBBA33D1F3CB
:10264000BB3391F3BC3231F40E94A12EBA2DB77086
:10265000D9F7EACFB23241F441914F3F59F34232B8
:1026600019F30E94A22EF8CFB134B0F0BB35A0F41C
:10267000B154BB0FB0936A01B081B13418F0BB35CF
:1026800008F40AC0F8D3DCE0C0E910916A01C10F78
:10269000D21DA993B993C8CF87E00895E9D38030BC
:1026A00009F0FFCA4A2F4B2BE1F340912201403041
:1026B000E1F3409122014030E1F71197F3CFD8D3F5
:1026C000A0932301B0932401EDCFB5D3A0912301B2
:1026D000A993A0912401A993E4CACAD34A2F0E94C6
:1026E0002B34C1D37C3221F4BDD30E949209F6CFA2
:1026F000D8CA0E943734A42FBB279DD3A993B9937E
:10270000D0CAF7018BD34A2FD73020F4C03D10F444
:102710000E94A639C6CAF70181D35A2FAC2FBD2F0C
:102720000E941A790E946E390E946E320E946E32A7
:102730000E946E32B6CA70910C0174FD30C098D3FD
:10274000A1B9AFCA70910C0174FD29C0F70166D31D
:10275000D030B1F4BC2FB770B39577276FE7A0FDE9
:1027600070E8A0FD6FEF77FB770F70F967FB660FDE
:1027700060F9BA95C1F702B1072B062302B991CAD5
:10278000D13041F4B2B1C095BC23C095CA23BC2B53
:10279000B2B987CAD230E9F70E94E41782CA82E24E
:1027A000089566D30E9423347CCA45D3C093700138
:1027B000D093710109911991105854D37C32A9F426
:1027C0002DD3B058D058C017D10710F00C2F1D2FA3
:1027D000A017B10710F40A2F1B2FD0917101C091DF
:1027E00070011058099319935CCA86E00895A0916E
:1027F0003E01A03011F08CE108951DD3C09370010B
:10280000D09371012FD37C3281F7FCD2C8ECD1E098
:102810007EE17B9FC00DD11DCA0FD21DBB27A881B1
:10282000D0917101C0917001A993B9933ACAA09156
:102830003E01A03011F08CE10895FDD2C0937001EB
:10284000D09371010FD37C3281F6DCD2C8ECD1E099
:102850007EE17B9FC00DD11DCA0FD21DA2EBCA0F16
:10286000A2E0DA0FBB27A881A695BA2FA777B29569
:10287000B078AB2BBB27D0917101C0917001A993A7
:10288000B9930FCA86E00895D6D2C0937001D09351
:102890007101E8D27C32B1F7B5D2C8ECD1E07091C9
:1028A0003E017370703021F5AF93BF93A695B69536
:1028B0007EE17B9FC00DD11DCA0FD21D7881BF91D3
:1028C000AF91A0FD7695B0FD7695B0FD7695A2EB23
:1028D000B2E0CA0FDB1FAC9170FDA295A695A77060
:1028E000BB27D0917101C0917001A993B993D9C947
:1028F0007130D1F4AF93A695A695A69575E17B9F0F
:10290000C00DD11DCA0FD21D7881AF91A2FD729565
:10291000A1FD7695A1FD7695A0FD76957170D1E02B
:10292000C72FA881A295DACF7130F1F7AF93A695A2
:10293000A6957EE17B9FC00DD11DCA0FD21D788167
:10294000AF91A1FD7295A0FD7695A0FD769573706F
:10295000D1E0C72FA881A295C1CFAF93A6957AE207
:102960007B9FC00DD11DCA0FD21D7881AF91A0FDF4
:102970007295A72FB3CFA0913E01A03011F08CE14A
:102980000895A3E0F1D1A33080F0A0915801B09157
:102990005901B33010F082E10895B23039F4A73F05
:1029A00028F082E1089581E208953BCACCE3DDE09E
:1029B000CA0FDB1FC0934601D0934901AC81A03000
:1029C00091F3AE3180F7BB81B03069F3B73158F77E
:1029D000C0915801D09159012596BA9F000C111C45
:1029E000000C111CC00DC11DD330E8F6D0915A0166
:1029F000C0915C01C0934801D0934B01CF3F51F08F
:102A0000DF3F41F0CA0FCA95CE3138F4DB0FDA95BB
:102A1000D73118F40E948D3743C986E10895A091FB
:102A20003E01A03011F08CE1089520D2A0912D013B
:102A3000A460A0932D0135C9A0912901A062A093A3
:102A400029012FC9A0912901AF7DA093290129C98E
:102A5000A3E08AD1A33009F0E4C90E944D2040339D
:102A600010F08EE108950E9461208030D9F718C9D6
:102A7000A3E07AD1A33009F0D4C90E944D2040339D
:102A800010F08EE108950E9464208030D9F708C9C3
:102A9000A3E06AD1A23019F0A33021F0C2C9A4E1A9
:102AA000A0935C010E945B20803009F4F9C808956E
:102AB0000E945E20803059F4F3C8A1E055D1A130C6
:102AC00009F0AFC90E944D20443191F38EE1089581
:102AD000A2E04AD1A23009F0A4C9A0915801B09156
:102AE000590140915A01CCE3DDE0403041F0D395EB
:102AF000413029F0D395423011F082E108950E94CF
:102B00000E3A0E94FD3A803009F00895C9C8A2E04B
:102B10002BD1A23009F085C9A0915801B09159017B
:102B200040915A01CCE3DDE0403041F0D395413093
:102B300029F0D395423011F082E108950E94C73AFE
:102B40000E942A3A803011F308954EC0F7013ED119
:102B5000A09374010E9424396830B9F790FF28C00F
:102B6000592F0E942639603481F7A030C9F0DDE08A
:102B7000CCE3409174014B0F4A1BC40FD21DA1300E
:102B800039F00E942A39603579F55883AA95EFCF3C
:102B90000E942F39683541F558830E94203981C839
:102BA0000E942A395030A1F350937401A52FDFCF32
:102BB000592F0E9426396831B9F43A2FDDE0CCE371
:102BC000409174014B0F4A1BC40FD21D58815030E5
:102BD00011F4303031F00E942639683229F4AA9578
:102BE00069F70E9420395DC88FE0089541D1A09314
:102BF0005801B093590137D17C3249F4319632D122
:102C0000723231F031970E94920985D1F4CF49C8D0
:102C10007191723231F07F3F21F0BB27A72F7BD11A
:102C2000F7CF7081E8CFA0913E01A03011F48DE183
:102C30000895A7E099D0B0915801B0934C01B130FC
:102C400039F0B23009F1B33009F43CC085E10895A0
:102C5000A730E1F7C8E5D1E0BA81B0934901BC8162
:102C6000B0934601BE81B0934A01B885B093470145
:102C7000BA85B0934B01BC85B09348010E94E534FE
:102C8000803009F008950CC8A63001F7C8E5D1E0FE
:102C9000BA81B0934901BC81B0934601BE81B09323
:102CA0004A01B885B0934701BA85B0934801BB8506
:102CB000B0934B010E94E534803009F008950C94E4
:102CC000500EC4CFA430E9F7C8E5D1E0BA81B09383
:102CD0004601BB81B0934901BC81B0934B01BE81D9
:102CE000B09348010E94E534803009F008950C94B7
:102CF000500EA0913E01A03011F08CE10895F70133
:102D00008DD0C0935801D093590150917401A517EB
:102D100008F45A2FA8E7B1E0503071F04D91A0931C
:102D20007501B0937601A42FBB27F5D0A091750152
:102D3000B09176015A95F0CFAA27BB27ECD00C941E
:102D4000510EA0913E01A03011F08CE10895A1E058
:102D50000BD0A13040F0A09158014A2F43700E943F
:102D60005B380C94500E5DC8F701A03009F408954B
:102D7000DF93CF93C8E5D1E040E05A2F503029F4DB
:102D8000A42F7F01CF91DF910895DF93CF934F93CD
:102D90005F930E9492095F914F91CF91DF918931AA
:102DA00021F488277F01A42F0895A993B99343950F
:102DB0005A95503019F371917032E9F37C3229F34E
:102DC0003197A42F7F01CF91DF910895A3E0CCDF4D
:102DD000A33009F590915801B0915A01A0915C017E
:102DE0000895D0915801C0915A01F0915C01E09191
:102DF0005E01C0934601D0934901E0934701F093EF
:102E00004A010895A2E0B1DFA23029F4B09158013F
:102E1000A0915A010895AF91AF9103C8A2E0A5DF38
:102E2000A230C9F7C0915801D0915901A0915A011F
:102E3000B0915B010895F70115D0713478F07B35BE
:102E400038F47154770FDCE0C0E9C70FD21D089544
:102E5000713620F07B3710F47156F4CF8F918F913B
:102E600087E0089571917032E9F30895F7010895AC
:102E7000F7010C949209EF93FF930E940333EC2F18
:102E8000FD2F00E00E94A33270912D01713011F4EA
:102E9000872F08C04A3EC9F400937401003031F412
:102EA000AA27BB278827FF91EF910895C8E7D1E0B3
:102EB000A191A9930A95E1F7A0E2A993AFEFA99395
:102EC000E8E7F1E00E949209EDCF4C3E49F4003072
:102ED000C9F2AA940E940333A0E2A8830A95D2CF34
:102EE000403248F24B3738F6AA2DAD3120F60E9419
:102EF000A22E0395C7CF92E0BB27AC2DA3950E94CD
:102F0000CB2D4AE30E94A22EBB27AD2D0E94CB2DD4
:102F10000E94A12E0895DF93CF93BF93AF93A0910A
:102F20005801B0915901B33098F4CCE3DDE0CA0FF9
:102F3000DB1FAF91BF91A883C0915801D091590177
:102F40002196C0935801D0935901CF91DF910895F4
:102F5000B45090F0AA0FBB1FB33070F4CCE3DDE0A7
:102F6000CA0FDB1FAF91BF91A993B993C0915801CC
:102F7000D09159012296E5CF82E1AF91BF91CF91D7
:102F8000DF91089570912C01A0FF0895A33059F4AA
:102F900050915C015F70550F707F572B70912C0121
:102FA00050932C01089550916001F4CF0E94672046
:102FB000403011F466270895409360010E94582024
:102FC000413009F066270895AF3F31F42C9A2CBCAC
:102FD000ACE5ACBD3DBC0895A7F92CBCAF73A064B3
:102FE000ACBD3DBCA5B1A4FBA5B90895BDB5B7FF67
:102FF000FDCF08955091720140917301433038F430
:10300000DDE0CCE3C50FD41FA991BB2710C0505001
:10301000444058F0550F441F433038F4DDE0CCE312
:10302000C50FD41FA991B99102C082E108954091C2
:10303000720150917301430D521D409372015093E0
:103040007301803009F408954F914F910895A0EADB
:10305000B1E04FEF52E24D935A95E9F7C8E9D1E05C
:1030600040E25A91503211F44A95D9F7442EA0EA21
:10307000B1E0C8E7D1E04C0EA03C28F4C41518F428
:103080004881403009F4089593D04F3FE1F37AD05E
:103090004F3FC9F3403081F798D0403069F73DD0B9
:1030A000403051F70AD0403039F74991413618F095
:1030B0004B3708F440524D93DFCF4881403320F026
:1030C0004A3310F4405302C044270895642F7727F1
:1030D00021964881403380F04A3370F44053660FA4
:1030E000771F0B01660F771F660F771F600D711D2D
:1030F000640F721D2196EDCF703029F04DE14D9394
:103100007D936D9308956A3020F04CE14D936D935B
:103110000895605D6D934CE108954881443211F04B
:103120004427089566277727219658815033F8F071
:103130005A3310F450530BC05134C8F0573410F4C4
:10314000575305C0513698F0573688F457555F707D
:103150005295550F661F771F550F661F771F550F26
:10316000661F771F550F661F771F2196DECF7030C1
:1031700029F04FE14D937D936D9308954EE14D936A
:103180006D9308954881423211F0442708952196A5
:103190004D934991423219F44D9341E008954030E6
:1031A00029F442E24D934FEF4D9308954D93F1CFA3
:1031B0004881473211F04427089521964D93499153
:1031C0004030E1F74FEF4D930895FF93EF93BF9396
:1031D000AF935F93E0E4F7E40E014591403089F04E
:1031E000689457E0A591AE3239F0B991B13608F044
:1031F000B052AB1709F0E8945A95A1F716F0E00128
:10320000EBCF5F91AF91BF91EF91FF91403041F0D3
:103210004D934F934881403211F42196FBCF4F914B
:103220000895CBE7D1E0A0EAB1E040E2E0E24993C3
:10323000EA95E9F7A097A03C29F04D91423010F0B3
:103240004F3F11F429920895403220F0403810F495
:1032500086D0F1CF4C3121F4ED91FF2719D0EBCF7F
:103260004D3121F4FD91ED9113D0E5CF4E3131F484
:1032700044E275D0ED91FF273CD0DDCF4F3131F4E2
:1032800044E26DD0FD91ED9134D0D5CF50D0D3CF65
:10329000E8944FE24395E051F742E0F7E05FF84DE4
:1032A000403311F063D068944FE24395E85EF340F9
:1032B000E0F7E851FC4F16F0403311F057D0689416
:1032C0004FE24395E456F040E0F7EC59FF4F16F01B
:1032D000403311F04BD068944FE24395EA50E8F741
:1032E000E65F16F0403309F041D040E34E0F3ED088
:1032F0000895E8944F2F42954F7011F012D06894C2
:103300004F2F4F700EF011F00CD068944E2F429555
:103310004F700EF011F005D068944E2F4F7001D011
:103320000895405D4A3308F0495F20D00895E0E4F5
:10333000F7E45591503009F40895451711F0379688
:10334000F8CF5F9357E045914E3209F00FD05A9570
:10335000D1F75F915C3110F040E208D008954993B5
:10336000CB3918F029924F914F9108954993CB3959
:1033700028F029924F914F914F914F910895FF93CB
:10338000EF93A0913E01A0936E01AA270E945B2DAE
:10339000A0912C01A0936A01A0910F01A0936D014F
:1033A000A0912A01A093690120922A01E8ECF1E0A2
:1033B000CCE2D7E0BEE2AEE141914993AA95E1F7B4
:1033C000BA95C9F7EF91FF910895FF93EF93A091FC
:1033D0006E010E945B2DA0916D01A0930F01A09141
:1033E0006A01A0932C01A0916901A0932A01ECE24B
:1033F000F7E0C8ECD1E0DECFA0910C01A4FD35C010
:10340000C6E0D4E0A9E4BFE441B158E040FDB9937F
:1034100040FFA99346955A95C9F7C4E2D4E0A0E3CA
:10342000B1E340B158E040FDB99340FFA993469500
:103430005A95C9F7C8EBD6E0AFEABFE241B158E010
:1034400040FDB99340FFA99346955A95C9F7C6ED3B
:10345000D6E0A0E8BEE440B158E040FDB99340FF9B
:10346000A99346955A95C9F708950E9430301300E4
:1034700020494F2044495341424C4544200008957F
:10348000452FA6E10E94AC2D4F5B0E94A22E4DE37A
:103490000E94A22EA7E10E94AC2DC0E9DCE0C50F7E
:1034A000D21DC50FD21DA991B9919DE00E94CB2DCF
:1034B0000895A3E10E944930A5E0C62FCA95AC9FAC
:1034C000CCEEDCE0C00DD11DA881A7FF0AC00E9490
:1034D0003030FF43414C4C202000A981AF770EC013
:1034E00008950E943030FF464F5220004A81469591
:1034F0004F5B0E94A22E0E94A12EA981BB27A395FB
:1035000092E00E94CB2D4AE30E94A22EBB27A88105
:103510000E94CB2D089520920F01A7E00E94AC2DB0
:103520000E943B2E0E94303012004249542030311C
:1035300032333435363700000E94303013004449AE
:1035400052000E94303014004C455600A7E20E9401
:10355000AC2D0E94303016002045786974200000A0
:10356000A0E60E94AC2D0E94303016062020476F46
:1035700020200000A0E40E94AC2D0E943030160CE8
:103580002053746570200000A7E10E94AC2D0E94BA
:10359000303016122056696577200000AEE6A09301
:1035A0002B07A7E30E94AC2D0E9430301618202074
:1035B00020202000A5E00E94AC2D0E9430300000A9
:1035C0004156522D43686970426173696332204DE0
:1035D0004F4E202020205000409137014F5C0E9428
:1035E000A22E0E943030FF3A000092E0BB27AC2DA3
:1035F000A3950E94CB2D0E943030FF3A0000BB27DC
:10360000AD2DA3950E94CB2DEBE7F1E0C6EED1E006
:10361000AEE141EFB191B03031F0BE8F4CAF499384
:10362000AA95C1F706C0B0E2BE8F4CAF4993AA95E8
:10363000D1F7A7E10E94AC2DC0E0D4E0E1E1F0E1D8
:103640000E9435319DE050E0452F4C5FB42FAA27F2
:103650000E94493015DF53955D30B1F7452F495031
:10366000B42FA9E00E9449300BDF53955A31B1F7CE
:10367000A7E30E94AC2DC3E1D4E0EDE1F0E10E94AC
:1036800035310E9430300413535441434B3A00000B
:103690009927BB27A0916F010E94CB2D6CE0C091B0
:1036A0006F01C61720F0C61BB4E0B60F02DF6A95A3
:1036B000B1F708954F935F936F937F93EF93FF93C9
:1036C000CF93DF93AF93BF93AF92BF928F939F93AC
:1036D00056DEA7DD20DF2ED08827A0912D014D3E9C
:1036E00011F4A16011C0413F11F4AA270DC0423F5F
:1036F00011F4A46009C0433F71F767DE0E9497325E
:10370000AA270E945B2DE6CFA0932D0140911601C0
:103710004030E1F75ADE9F918F91BF90AF90BF91FB
:10372000AF91DF91CF91FF91EF917F916F915F9179
:103730004F910895209217015FDE409117014030AC
:10374000D9F30C943B3320922A0120923E01A5E04C
:103750000E94AC2DC0E0D0E0EDE1F6E10E94D33153
:10376000A0E50E94AC2D0E943030010244464C413D
:1037700053482073697A653A20000E9467204F37CA
:1037800049F40E943030FF353132204B6942797460
:10379000650011C04F3F41F40E943030FF31204D91
:1037A00069427974650007C00E943030FF302042C2
:1037B0007974650013C00E9458204130D1F0E2EEC8
:1037C000F9E3E8940E945E34413009F434C0443097
:1037D00009F4B9CF423099F733D0B5CFEEE1FAE32F
:1037E000E8940E945E34413009F425C04430B1F7BA
:1037F000AACFE6EAF9E3E8940E945E34413009F486
:103800001AC0473019F40E942D1D9DCF4A3011F483
:1038100017D099CF423011F46DD095CF433019F4C1
:103820000E94841D90CF443019F40E94D61D8BCF86
:103830004530F9F688CFA0911601A030E1F7089540
:103840000E940E374F466F726D6174204D6564693A
:10385000756D3F00413009F00895A6E20E94AC2D3D
:10386000C2E0D8E0EBE1FCE00E949B310E943030E6
:103870000903466F726D617474696E672E2E2E2077
:103880002020202020000E9430300B0300000E94E6
:103890006A20803001F50E9430300903466F726D56
:1038A000617474696E672E2E2E20446F6E65210040
:1038B000A2E70E94AC2D0E9430300B032020205044
:1038C0007265737320616E79206B65792120200009
:1038D0000E94973208950E9430300903466F726D3E
:1038E000617474696E672E2E2E204572726F72217C
:1038F0000000DECFA0E60E94AC2DC4E0D8E0E9E1F4
:10390000FDE00E949B310E943030090541766169DB
:103910006C61626C653A00000E9430300A054669AD
:103920006C65733A20009CE00E944A20DF93CF939D
:10393000DF010E94CB2D0E943030FF202F000E941B
:103940006720A42FB0E011960E94CB2D0E9430304A
:103950000B05426C6F636B733A00AF91BF910E948D
:10396000CB2D0E943030FF202F000E945220A0EF6C
:10397000A49FD0011197B03009F413970E94CB2D6A
:10398000A6E00E94AC2D0E9430300C052020205073
:103990007265737320616E79206B65792120200038
:1039A0000E949732089520457869742020496E66F8
:1039B0006F204261636B7570526573746F725265EC
:1039C0007363616E20202020202044656C6574653F
:1039D000202020202020202020202020466F726DD3
:1039E0006174204578697420466F726D617420207F
:1039F0002020202020202020202052657363616E2B
:103A000020202020202020202020202020202020B6
:103A10002020202020202020202020202020204581
:103A200078697420202020202020202020202020A1
:103A300020202020202052657363616E20202020EA
:103A40002020202020202020202020202020202076
:103A50002020202020202020202077270BD1A4E028
:103A60000E94AC2DC1E0D2E0ECE1F5E10E94D3313F
:103A7000A0E40E94AC2D0E943030030244656C65C6
:103A800074652066696C6500B0D07093580105D3E9
:103A90004C3FD1F34CD1413019F4A72FB7D20ED3FC
:103AA00008957727E7D0A4E00E94AC2DC1E0D2E0D2
:103AB000ECE1F5E10E94D331A0E40E94AC2DA0E13D
:103AC000A0935C010E943030030253617665205060
:103AD0000000C7D28AD070935801DFD2403E20F454
:103AE000403161F0F4D0DECFD5D2D03021F4CC30EB
:103AF00010F427D1D7CF8AD2B4D108950CD1413058
:103B000089F684D2BAD108957727B4D0A4E00E9470
:103B1000AC2DC1E0D2E0ECE1F5E10E94D331A0E4AC
:103B20000E94AC2DA2E1A0935C010E943030030200
:103B30004261636B7570000058D070935801ADD22C
:103B4000403920F4423161F0C2D0DFCFA3D2D0306F
:103B500021F4C03610F4F5D0D8CF58D21CD2089535
:103B6000DAD0413091F652D222D20895772782D00E
:103B7000A4E00E94AC2DC1E0D2E0ECE1F5E10E94AE
:103B8000D331A0E40E94AC2D0E94303003024C6F70
:103B900061642050000065D228D0709358017DD216
:103BA000403111F0A2D0E3CF88D10895772762D0B9
:103BB000A4E00E94AC2DC1E0D2E0ECE1F6E10E946D
:103BC000D331A0E40E94AC2D0E9430300302526534
:103BD00073746F72650009D0709358015ED24231E0
:103BE00011F08ED0E4CFFBD108957727B5D00BD15B
:103BF0000E9497324D3E21F42FD14F914F9108955D
:103C00004A3E09F40895403E19F40FD17727EECFCC
:103C1000413E21F40AD170916001E8CF443E49F45D
:103C2000703031F302D17150472F4F704F30F1F2A5
:103C3000DECF453E59F440916001471709F4D8CFD3
:103C4000F4D07395472F4F7089F2D1CF463E29F4B7
:103C5000703170F2EAD07051C9CF473E51F44091B3
:103C600060014F3031F04051471718F0DED0705FDF
:103C7000BDCFBECF0E946720403019F44F914F91C5
:103C80001BC0409360010E946E320E946E3210D2BF
:103C9000413019F04F914F9101C008950E94E536CF
:103CA0004F44464C415348206E6F7420666F726DCE
:103CB00061747465640008950E94E5364F44464C73
:103CC000415348206572726F7221000008950E946E
:103CD000E5364F43616E206E6F7420736176652008
:103CE0006F6E20746869730008950E94E5364F4E28
:103CF0006F2042415349432066696C650000089576
:103D00000E94E5364F4E6F204241434B555020668E
:103D1000696C650008950E940E37C04F7665727712
:103D2000726974652066696C653F000008950E94A1
:103D30000E374F44656C6574652066696C653F009D
:103D400008950E94E5364F4E6F20737061636520C1
:103D50006C656674000008955F936F937F93A72F3F
:103D6000A07FA0936C01A0916C01AF70AB5FBA2FE4
:103D7000A4E00E944930A6E00E94AC2DA0916C0105
:103D8000BB2795E00E94CB2D0E94A12EA5E00E94AA
:103D9000AC2DA0916C01A09358017FD1ADD04F3FC5
:103DA00061F1A0916C01A093580140E040935A0149
:103DB00042E040935C01882784D1803091F4CCE3C9
:103DC000DFE00E94A12E5CE05F934991403808F04B
:103DD0004EE2403208F440E20E94A22E5F915A95D2
:103DE00099F7A0916C01A395A0936C01AF7009F0B5
:103DF000BACF7F916F915F9108955DE00E94A12EEF
:103E00005A95E1F7EECF4F935F93C4E1D5E0472F8A
:103E10004F705EE1459FC00DD11D52EF47E15993B0
:103E20004A95E9F75F914F9108954F935F93C4E1ED
:103E3000D5E0472F4F705EE1459FC00DD11D5CE07E
:103E400044E059934A95E9F75AE043E159934A957A
:103E5000E9F75F914F910895A0911601A030E1F725
:103E60000895709358014CE040935A0140E140930B
:103E70005C0121D1803009F01FCF709358019091DF
:103E80003D01E0E0F0E99770929540EC949FE00DE1
:103E9000F11D40E04F9300E0CCE3DFE01591199372
:103EA0000A95E1F740935A0142E040935C010CD13E
:103EB0004F9143954C3071F7089590913D01977063
:103EC000E0E0F0E9929540EC949FE00DF11D40E0B8
:103ED0004F9340935A0142E040935C017093580124
:103EE000F0D0CCE3DFE00E947A7932964F9143958F
:103EF0004C3071F778940895403139F40E94303095
:103F0000FF4241533A0040E10895423139F40E94A2
:103F10003030FF4255503A0042E10895443139F4BF
:103F20000E943030FF5553523A0044E10895463123
:103F300039F40E943030FF4348383A0046E1089592
:103F4000483139F40E943030FF4156523A0048E17E
:103F500008954A3139F40E943030FF47504F3A00FB
:103F60004AE108954C3139F40E943030FF53414DFD
:103F70003A004CE108954E3139F40E943030FF4C44
:103F8000424C3A004EE108950E943030FF2D2D2D15
:103F90002D004FEF08957093580140E640935A0169
:103FA00042E140935C0187D0803009F085CE709368
:103FB00058014427E0E0F0E94F93CCE3DFE0002430
:103FC000159019920A94E1F740935A0142E0409308
:103FD0005C017AD04F914395403671F7089540E0E7
:103FE000E0E0F0E94F9340935A0142E040935C01D6
:103FF0007093580166D0CCE3DFE00E947A79329664
:104000004F914395403671F7789408954F93FF93FD
:10401000EF93DF93CF93BF93AF9340912C014093E5
:1040200061014CE440932C01C6E0DAE0E7E1FCE0FA
:104030000E949B310E9430300B0757726974696E81
:104040006720646174612E2E2E00409161014093BF
:104050002C01AF91BF91CF91DF91EF91FF914F91E3
:104060000895CAE2CAE240913D01942F4F5C499302
:1040700040E249934BE54993409129014F934068B1
:10408000409329010E94AC794DE549934F914093AB
:10409000290108950E94AF3B08950E947B3C0E9435
:1040A0003E3A08950E94EB3908950E946B3A0895B4
:1040B0000E948A3B08950E94103C08950E94833C10
:1040C00008950E94033D08950E94A43C08950E9413
:1040D000F93908950E941C3B0895A1E00E94233401
:1040E00020922A0120923E01A7E00E94AC2DC0E060
:1040F000D0E0EDE1F6E10E94D331A0E70E94AC2DC3
:104100000E94303001024156522D4368697042616D
:104110007369633220636F6E6669677061676500FB
:10412000A7E00E94AC2D0E94303014014368656303
:104130006B73756D3A20000049D150D084D0B6D051
:10414000E7D018D1EEE2F4E4E8940E945E34413006
:1041500009F437C1423059F440910C0151E0452730
:1041600040930C010E9407790E94E121E6CF433081
:1041700059F440910C0152E0452740930C010E94F4
:1041800007790E94E121D9CF443059F440910C01C4
:1041900054E0452740930C010E9407790E94E121D9
:1041A000CCCF453059F440910C0158E0452740935D
:1041B0000C010E9407790E94E121BFCF473049F4EA
:1041C0000E941A79439547700E9415790E94E12157
:1041D000B4CF4A3011F40E94272A7FCFA6E00E9474
:1041E000AC2D0E94303003014B6579626F617264BF
:1041F000206C61796F75743A0000A7E040910C0162
:10420000417009F4A1E70E94AC2D0E9430300312E6
:104210004445202851574552545A2900A7E040915F
:104220000C01417009F0A1E70E94AC2D0E943030D2
:104230000412555320285157455254592900A7E0DC
:104240000E94AC2D0895A6E00E94AC2D0E94303053
:10425000060153657269616C2073706565643A008C
:10426000A7E040910C01427009F4A1E70E94AC2D37
:104270000E943030061220313230302042707320DC
:104280002000A7E040910C01427009F0A1E70E94D4
:10429000AC2D0E9430300712203234303020427072
:1042A00073202000A7E00E94AC2D0895A6E00E9494
:1042B000AC2D0E943030090149324320737065658E
:1042C000643A0000A7E040910C01447009F4A1E7B2
:1042D0000E94AC2D0E943030091220203130302055
:1042E0006B487A202000A7E040910C01447009F04F
:1042F000A1E70E94AC2D0E9430300A1220203430F9
:1043000030206B487A202000A7E00E94AC2D089551
:10431000A6E00E94AC2D0E9430300C015350492081
:1043200073706565643A0000A7E040910C01487025
:1043300009F4A1E70E94AC2D0E9430300C1220201D
:10434000202035204D487A202000A7E040910C0124
:10435000487009F0A1E70E94AC2D0E9430300D1288
:104360002020313536206B487A202000A7E00E94BB
:10437000AC2D0895A6E00E94AC2D0E9430300F01B4
:10438000454550524F4D20616464726573733A0025
:10439000A1E70E94AC2D0E9430300F122020202077
:1043A00020000E941A794770405D0E94A22E0E9450
:1043B0003030FF20202020200000A0E70E94AC2DFC
:1043C0000895A0911601A030E1F70895AA27BB2710
:1043D000CC27DD27EE27FF27159042E0149EA00D85
:1043E000B11DC21DD21D459147E0149EA00DB11D07
:1043F000C21DD21DFE3881F7EE27F0EF459141E74F
:10440000149EB01DC11DD21D459147E0149EB01DE4
:10441000C11DD21DF03091F7BF93AF93DE019FE035
:104420000E94262EAF91BF910E94262E089520450E
:1044300078697420204B65796220205365722020B2
:104440002049324320202053504920202020202082
:104450002020454550524F4D202020202020202054
:1044600020202020436C6F6E6520AEE0A0932C01CD
:10447000C1E0D4E0ECE1F1E10E949B310E943030D8
:10448000050500000E94F8010E94303006032863F1
:104490002920323030362D38204A6F657267205718
:1044A0006F6C6672616D0000A2EAA0932C010E94FD
:1044B0003030080320202020202044656469636197
:1044C00074656420746F20202020202000000E944A
:1044D00030300903466C6F7269616E2C2045726939
:1044E0006B20616E64204469616E612E0000AEE055
:1044F000A0932C010E9430300B0254686973207322
:104500006F667477617265206973206C6963656E8C
:10451000736564000E9430300C04756E646572200F
:10452000746865207465726D73206F6620746865A9
:1045300020000E9430300D04474E55205055424C0B
:104540004943204C4943454E534520562E322000C6
:104550000E9430300E035573652069742061742009
:10456000796F7572206F776E207269736B2100000E
:10457000A2ECA0932C010E9430301007205052452D
:10458000535320414E59204B455920000E949732E9
:10459000089561E00E944734509116015D3E09F490
:1045A00008954531B1F790913D01E0E0F0E9977051
:1045B000929540EC949FE00DF11DCCE3DDE050E0DE
:1045C000459149935A95E1F7CCE3DDE00E94033928
:1045D0000E944734509116015D3E11F34630A1F719
:1045E0006395CCEBDDE00E9403390E944734509183
:1045F00016015D3EA9F24630A1F763956931E9F6EF
:1046000044E00E942B34089590913D019770E0E0C2
:10461000F0E9929540EC949FE00DF11D45E10E9478
:104620002B3460E06F93CCE3DFE00E94E038803011
:1046300041F0813051F1883241F145E10E942B3443
:10464000F2CF46E00E942B34CCEBDFE00E94E03852
:10465000803041F08130C9F08832B9F045E10E94E4
:104660002B34F2CF0E947A797894329646E00E94F9
:104670002B346F9163956C30A9F60E943734443027
:10468000E1F746E00E942B3408956F91089561E0B0
:104690000E944734509116015D3E09F4089545315A
:1046A000B1F7A0E8762F7A95A79FE001ACE3BDE0D3
:1046B00070E80E949D394D937A95D9F7CCE3DDE0FF
:1046C0000E9403390E944734509116015D3E31F338
:1046D0004630A1F763956F3021F744E00E942B34F8
:1046E000089545E10E942B3460E06F93CCE3DDE058
:1046F0000E94E038803031F0883201F145E10E94BB
:104700002B34F4CFA0E8762F7A95A79FE001ACE395
:10471000BDE070E84D910E94A6397A95D9F746E040
:104720000E942B346F9163956E30F9F60E943734F6
:104730004430E1F746E00E942B3408956F910895CC
:1047400002414253282E2E2E0353474E282E2E2E42
:1047500004535152282E2E2E054E4F54282E2E2E05
:1047600006524E44282E2E2E07414443282E2E2E2C
:1047700008494E282E2E2E2E09585045454B282EDE
:104780000A54454D50282E2E0B4C4F282E2E2E2EDF
:104790000C4849282E2E2E2E0D4B4559282E2E2EF4
:1047A0000E455045454B282E0F455252282E2E2E91
:1047B000104152282E2E2E2E1153494E282E2E2EC9
:1047C00012434F53282E2E2E134654595045282E4F
:1047D000144653495A45282E155053544154282EF7
:1047E00016535049282E2E2E174D454E55282E2E45
:1047F000805052494E542E2E81434C532E2E2E2E35
:1048000082474F544F2E2E2E83424F582E2E2E2E3F
:104810008441434F50592E2E8553594E432E2E2EF0
:1048200086454E442E2E2E2E8742434F50592E2E13
:10483000885448454E2E2E2E89504F532E2E2E2E04
:104840008A4E4F54452E2E2E8B454D49542E2E2EDA
:104850008C52524541442E2E8D5257524954452E6A
:104860008E474F5355422E2E8F52455455524E2E41
:1048700090564D4F44452E2E914E4558542E2E2E77
:1048800092494E5055542E2E93504C4F542E2E2E4E
:1048900094574149542E2E2E95545345542E2E2E66
:1048A00096544745542E2E2E974653454C45435417
:1048B000984F4E4552522E2E99535055542E2E2E0F
:1048C0009A534745542E2E2E9B45504F4B452E2E26
:1048D0009C4745545049582E9D434952434C452EC0
:1048E0009E434F4C4F522E2E9F424F524445522EC4
:1048F000A0464F4E542E2E2EA150554D502E2E2EEA
:10490000A258504F4B452E2EA359454D49542E2E9B
:10491000A44C494D49542E2EA54745544348415275
:10492000A644524157544F2EA7504C41592E2E2E7B
:10493000A85350524954452EA95343524F4C4C2E24
:10494000AA425245414B2E2EAB464153542E2E2E99
:10495000AC534C4F572E2E2EAD445241572E2E2E77
:10496000AE49434F4D4D2E2EAF444154412E2E2E75
:10497000B043544558542E2EB146524541442E2E34
:10498000B24657524954452EB343424F582E2E2E0D
:10499000B447455441545452B54644454C4554459A
:1049A000B646424F582E2E2EB750414C45545445D2
:1049B000B8464F522E2E2E2EB949462E2E2E2E2E72
:1049C000BA4449522E2E2E2EBB4F55542E2E2E2E2B
:1049D000BC46434952434C45BD414C4552542E2E92
:1049E000BE46435245415445BF41534B2E2E2E2EB9
:1049F000C03F2E2E2E2E2E2EC742432E2E2E2E2E72
:104A0000CA4E4F2E2E2E2E2ECB454D2E2E2E2E2E16
:104A1000CC5252442E2E2E2ECD5257522E2E2E2EAA
:104A2000CE474F532E2E2E2ECF5245542E2E2E2EA5
:104A3000C2474F2E2E2E2E2ED0564D2E2E2E2E2EDF
:104A4000D2494E502E2E2E2ED3504C2E2E2E2E2EA0
:104A5000D74653454C2E2E2EDC4750582E2E2E2E48
:104A6000DD43492E2E2E2E2EDE434F4C2E2E2E2E83
:104A7000DF424F2E2E2E2E2EE44C494D2E2E2E2E62
:104A8000E54743482E2E2E2EE644544F2E2E2E2E32
:104A9000E85350522E2E2E2EED44522E2E2E2E2E18
:104AA000EE49432E2E2E2E2EEF44412E2E2E2E2E4C
:104AB000F14652442E2E2E2EF24657522E2E2E2ED8
:104AC000F44741542E2E2E2EF54644454C2E2E2EC4
:104AD000F750414C2E2E2E2EFC4643492E2E2E2EC4
:104AE000FE4643522E2E2E2E002E2E2E2E2E2E2EF3
:104AF000A0910801B0910901ED01E2EBF2E0CE0FC7
:104B0000DF1FF6EFE0910E01FE0F7F934F92EEE173
:104B10004E2E6991ED915491762F7295762757FD1F
:104B2000672768B9ED91000056FD76B9049055FDF0
:104B300076B96991162E54FD76B91294162653FD56
:104B400076B907FC61254A9452FD76B9502D712D36
:104B500041F760910F0168B94F907F91EE91F0910C
:104B60000E01F395FA3029F4FF27A0930801B093C2
:104B70000901F0930E010C945E2CA0910801B091F4
:104B80000901D0910001C0910101C295DC0FDE7EC8
:104B9000E5E110900F01FD914D2FF0FD429548B9D0
:104BA00000004D2FF1FD429548B900004D2FF2FD58
:104BB000429548B900004D2FF3FD4295000048B9D9
:104BC0006D2F4D2FF4FD429548B9CD91F5FD6295BD
:104BD0005D2F68B9F6FD52956D2F4D2F58B9F7FD31
:104BE0006295C0FD4295000068B9FC2FEA95B9F6C0
:104BF00018B8EE91F0910E01F395F23029F4FF27E9
:104C0000A0930801B0930901F0930E010C945E2C5F
:104C1000A0910801B0910901D1E0FEE110900F01CF
:104C2000ED91CE2FC370588158B9CE2FC695C69539
:104C3000C3705881E29558B9CE2FC3705881CE2FDA
:104C4000C69558B9C695C3705881ED91CE2F58B905
:104C5000C3705881FA9541F718B8EE91F0910E01A2
:104C6000F395F33029F4FF27A0930801B0930901CD
:104C7000F0930E010C945E2CA0910801B0910901F3
:104C80000F9310900F01EAE2D1E0CD91C6950C2F61
:104C9000C295C770F881F8B9C02F0000C770F881BD
:104CA000000000000000F8B9CD91C6950C2FC29508
:104CB000C770F881EA9579F718B811970F91F091BC
:104CC0000E01F395F43029F4FF27A0930801B09367
:104CD0000901F0930E010C945E2CA0910801B09193
:104CE0000901D0910001C0910101C295DC0FDE7E67
:104CF000E0E110900F01FD914D2FF0FD429548B974
:104D00000000000000004D2FF1FD429548B9000061
:104D1000000000004D2FF2FD429548B90000000050
:104D20004D2FF3FD4295000048B9000000006D2FA3
:104D30004D2FF4FD429548B90000CD91F5FD6295E7
:104D40005D2F68B900000000F6FD52956D2F4D2FC4
:104D500058B9F7FD6295C0FD42950000000068B9A2
:104D6000FC2F00000000EA9551F6000018B8EE9103
:104D7000F0910E01F395F33029F4FF27A093080179
:104D8000B0930901F0930E010C945E2CA0910801E0
:104D9000B0910901C0914101D82DF6EFE0910E01CB
:104DA000FE0FE395E0930E01EA3088F1EC3069F5EF
:104DB0009396A0930801B093090120920E01DC3074
:104DC00031F4D0914001D09341010C945E2CD83144
:104DD00089F4A1E3B2E0C0912E01D3E2CD9FA00DF2
:104DE000B11DCFE0A0930801B0930901C093410128
:104DF0000C945E2CD83D49F4CBE4AEE0B2E0A09335
:104E00000801B0930901C09341010C945E2C0F93EB
:104E10001F932F93D83D28F4DC2F0C2F1C2F2C2F01
:104E200005C029E61DE208E8DCECCBE46C2F7C2F02
:104E30007295ED91E7FD6727EF775491ED9168B991
:104E4000172E56FD16B86C2F7C2F729555FD16B88F
:104E5000E7FD672754FD16B8EF77000053FD16B83D
:104E6000049052FD16B8502DED9168B9172E56FDDD
:104E700016B86C2F7C2F729555FD16B8E7FD672785
:104E800054FD16B8EF77000053FD16B8049052FD9C
:104E900016B8502DED9168B9172E56FD16B86C2F27
:104EA0007C2F729555FD16B8E7FD672754FD16B89F
:104EB000EF77000053FD16B8049052FD16B8502D40
:104EC000ED9168B9172E56FD16B86C2F7C2F729590
:104ED00055FD16B8E7FD672754FD16B8EF770000BB
:104EE00053FD16B8049052FD16B8502DED9168B9D7
:104EF000172E56FD16B86C2F7C2F729555FD16B8DF
:104F0000E7FD672754FD16B8EF77000053FD16B88C
:104F1000049052FD16B8502DED9168B9172E56FD2C
:104F200016B86C2F7C2F729555FD16B8E7FD6727D4
:104F300054FD16B8EF77000053FD16B8049052FDEB
:104F400016B8502DED9168B9172E56FD16B86D2F75
:104F50007D2F729555FD16B8E7FD672754FD16B8ED
:104F6000EF77000053FD16B8049052FD16B8502D8F
:104F7000ED9168B9172E56FD16B86D2F7D2F7295DD
:104F800055FD16B8E7FD672754FD16B8EF7700000A
:104F900053FD16B8049052FD16B8502DED9168B926
:104FA000172E56FD16B86D2F7D2F729555FD16B82C
:104FB000E7FD672754FD16B8EF77000053FD16B8DC
:104FC000049052FD16B8502DED9168B9172E56FD7C
:104FD00016B86D2F7D2F729555FD16B8E7FD672722
:104FE00054FD16B8EF77000053FD16B8049052FD3B
:104FF00016B8502DED9168B9172E56FD16B86D2FC5
:105000007D2F729555FD16B8E7FD672754FD16B83C
:10501000EF77000053FD16B8049052FD16B8502DDE
:10502000ED9168B9172E56FD16B86D2F7D2F72952C
:1050300055FD16B8E7FD672754FD16B8EF77000059
:1050400053FD16B8049052FD16B8502DED9168B975
:10505000172E56FD16B86D2F7D2F729555FD16B87B
:10506000E7FD672754FD16B8EF77000053FD16B82B
:10507000049052FD16B8502DED9168B9172E56FDCB
:1050800016B8602F702F729555FD16B8E7FD67278B
:1050900054FD16B8EF77000053FD16B8049052FD8A
:1050A00016B8502DED9168B9172E56FD16B8602F21
:1050B000702F729555FD16B8E7FD672754FD16B899
:1050C000EF77000053FD16B8049052FD16B8502D2E
:1050D000ED9168B9172E56FD16B8602F702F729596
:1050E00055FD16B8E7FD672754FD16B8EF770000A9
:1050F00053FD16B8049052FD16B8502DED9168B9C5
:10510000172E56FD16B8602F702F729555FD16B8E4
:10511000E7FD672754FD16B8EF77000053FD16B87A
:10512000049052FD16B8502DED9168B9172E56FD1A
:1051300016B8602F702F729555FD16B8E7FD6727DA
:1051400054FD16B8EF77000053FD16B8049052FDD9
:1051500016B8502DED9168B9172E56FD16B8602F70
:10516000702F729555FD16B8E7FD672754FD16B8E8
:10517000EF77000053FD16B8049052FD16B8502D7D
:10518000ED9168B9172E56FD16B8612F712F7295E3
:1051900055FD16B8E7FD672754FD16B8EF770000F8
:1051A00053FD16B8049052FD16B8502DED9168B914
:1051B000172E56FD16B8612F712F729555FD16B832
:1051C000E7FD672754FD16B8EF77000053FD16B8CA
:1051D000049052FD16B8502DED9168B9172E56FD6A
:1051E00016B8612F712F729555FD16B8E7FD672728
:1051F00054FD16B8EF77000053FD16B8049052FD29
:1052000016B8502DED9168B9172E56FD16B8612FBE
:10521000712F729555FD16B8E7FD672754FD16B836
:10522000EF77000053FD16B8049052FD16B8502DCC
:10523000ED9168B9172E56FD16B8612F712F729532
:1052400055FD16B8E7FD672754FD16B8EF77000047
:1052500053FD16B8049052FD16B8502DED9168B963
:10526000172E56FD16B8612F712F729555FD16B881
:10527000E7FD672754FD16B8EF77000053FD16B819
:10528000049052FD16B8502DED9168B9172E56FDB9
:1052900016B8612F712F729555FD16B8E7FD672777
:1052A00054FD16B8EF77000053FD16B8049052FD78
:1052B00016B8502DED9168B9172E56FD16B8612F0E
:1052C000712F729555FD16B8E7FD672754FD16B886
:1052D000EF77000053FD16B8049052FD16B8502D1C
:1052E000ED9168B9172E56FD16B8622F722F729580
:1052F00055FD16B8E7FD672754FD16B8EF77000097
:1053000053FD16B8049052FD16B8502DED9168B9B2
:10531000172E56FD16B8622F722F729555FD16B8CE
:10532000E7FD672754FD16B8EF77000053FD16B868
:10533000049052FD16B8502DED9168B9172E56FD08
:1053400016B8622F722F729555FD16B8E7FD6727C4
:1053500054FD16B8EF77000053FD16B8049052FDC7
:1053600016B8502DED9168B9172E56FD16B8622F5C
:10537000722F729555FD16B8E7FD672754FD16B8D4
:10538000EF77000053FD16B8049052FD16B8502D6B
:10539000ED9168B9172E56FD16B8622F722F7295CF
:1053A00055FD16B8E7FD672754FD16B8EF770000E6
:1053B00053FD16B8049052FD16B8502DED9168B902
:1053C000172E56FD16B8622F722F729555FD16B81E
:1053D000E7FD672754FD16B8EF77000053FD16B8B8
:1053E000049052FD16B8502DED9168B9172E56FD58
:1053F00016B8622F722F729555FD16B8E7FD672714
:1054000054FD16B8EF77000053FD16B8049052FD16
:1054100016B8502DED9168B9172E56FD16B8622FAB
:10542000722F729555FD16B8E7FD672754FD16B823
:10543000EF77000053FD16B8049052FD16B8502DBA
:10544000ED9128B82F911F910F910C945E2C0E9422
:105450000E376F436C6F6E652073797374656D3FA3
:105460002000413009F0089565D087D0803079F070
:1054700078D00E94E5364F4E6F20636F6E74726F66
:105480006C6C657220666F756E64200008958DD017
:10549000803069F066D00E94E5364F4E6F204D6532
:1054A000676136343420666F756E64000895CBD022
:1054B0009BD0EE27FF2750E060E00590B6D0059026
:1054C000BBD063956038C9F79CD05395A9F74CEAD7
:1054D0004ED040EA4CD04AD046EE49D00E946E32BF
:1054E0000E946E320E946E324CEA41D048EA3FD0B0
:1054F0003DD041ED3CD00E946E320E946E320E943F
:105500006E324CEA34D044EA32D030D04CEF2FD057
:105510000E946E320E946E320E946E3222D00E9431
:10552000E5368053797374656D20636C6F6E6564C6
:105530000000089543E54CBD2DBC249A2C984FEFF4
:105540004A95F1F72C9A4FEF4A95F1F72C984FEFC7
:105550004A95F1F72C984FEF4A95F1F70E946E3279
:1055600008952C9A4CE54CBD3DBC089544274EBD92
:105570004DB547FFFDCF4EB5089588274CEAF7DFBC
:1055800043E5F5DFF3DF433509F081E0EFDF089510
:10559000BF93AF934F93A42FBB270E94262E0E9448
:1055A000A12E4F91AF91BF910895882740E3DFDF8F
:1055B000DDDF40E0DCDFDADF4E3111F082E008951C
:1055C00040E3D5DFD3DF41E0D2DFD0DF463911F051
:1055D00082E0089540E3CBDFC9DF42E0C8DFC6DFE9
:1055E000493009F082E008954CEAC1DF40E8BFDFAE
:1055F000BDDFBCDF0E946E320E946E320E946E32AE
:1056000008954CE4B4DF452F4695B1DF452F440F94
:10561000440F440F440F440F440F440FA8DFA6DF8C
:105620000E946E320E946E32089540E4A0DF9EDF39
:10563000462F9DDF402D9BCF48E499DF97DF462F13
:1056400096DF402D94CF4F93FF93EF93DF93CF934B
:10565000BF93AF9340912C01409361014CE4409380
:105660002C01C5E0DAE0E8E1FCE00E949B310E94F9
:1056700030300B06436C6F6E696E6720537973741C
:10568000656D2E2E2E004091610140932C01AF914B
:10569000BF91CF91DF91EF91FF914F91089528B87D
:1056A00018954F935F936F93FF93EF93DF93CF938F
:1056B000BF93AF930F921F92FFB7FF9330921101E8
:1056C000B0913101B7FF5C98B7FD5C9A4B99BE7FF2
:1056D0004B9BB160B0933101C8E0D1E05F89A889EC
:1056E000E9890A881B88A00DE11DA88BE98BFFA121
:1056F0004491AD89AF3F09F4452F5AA54503B0E861
:10570000B10DB093B300EE89FF89488D598DAA275A
:10571000E2FDA095E5FDA095F4FDA09557FDA095AF
:10572000AA1FEE1FFF1F441F551FEE8BFF8B488FD4
:10573000598F830C921CEBA9FF81EF23E8B9789471
:10574000E9A190FC04C0F8A58F1608F490C0FCE015
:10575000E2FFFDEE8F1639F45E98E3FFAFC0B2E8CA
:10576000B0938000ABC0F1E1E2FFF3EF8F1639F4A4
:105770005E9AE3FFA3C0B2ECB09380009FC0FBE150
:10578000E2FFFFEF8F1621F4EFEFE0933B0196C0AD
:10579000F2E0E2FFF9EE8F1619F420923B018EC081
:1057A000F9E3E2FFF7E08F1609F088C0A8ECA883C0
:1057B000A1E0A9832E8288249924AAE0A9AFA5E0BC
:1057C000E2FFA39542E3E2FF4CE3BA8DB395BA172B
:1057D00031F4BB27EB8DFC8D3196EB8FFC8FBA8FAC
:1057E000E885E395E41709F4EE27E887FDE8E0E0B3
:1057F000AC89EA0FF21DB491B21511F0A395AC8BF0
:10580000BAA7A0915001A03009F458C0B09151013D
:10581000B395B0935101BA17C0F3BB27B0935101B0
:10582000E0915201F0915301C0915601D09157017E
:105830002196A191E0935201F0935301AE3F09F0FC
:1058400056D6FD1798F0EC1788F0A0913301A130DF
:1058500029F4A2E020925001A0933301E091540179
:10586000F0915501E0935201F093530127C0A091AC
:105870008400AA3FE0F3AB3F00F0AC3F00F0AD3F47
:1058800000F0AE3F00F0E5FD19C0E0912901E7FD11
:105890000C94C626E0913E01E53011F40C946D267F
:1058A000E37011F40C947825E13011F40C94BD25CB
:1058B000E23011F40C9408260C943C26A0911401BB
:1058C000A5FD23C0E091C000E7FF65C0E091C600E0
:1058D000F5EFB491B0FF34C0A7FF03C020921601CA
:1058E00057C0E33809F4E0E1F6E840910C0140FDCF
:1058F000FE5FEF77A4FFA6FDF395A4FFA0FDE0688F
:10590000E491E0931501A06244C0E0911501E09399
:105910001601E0931701EE3E19F4A2FD0C94380035
:1059200040912D01E33611F4A2FD4160E03711F4FE
:10593000A3FD4260EC3F09F4446040932D0128C070
:10594000E03F11F4A06825C0E03E11F4A06421C03E
:10595000E23121F4A160A7FDAE7F1AC0E93521F440
:10596000A260A7FDAD7F14C0E43151F4A6FD04C0D0
:10597000A460A7FDAB7F0CC0A860A7FDA77F08C0EF
:10598000E13121F4A061A7FDAF7E02C02092160193
:10599000AF71A093140140910C0141FD0E94A178C8
:1059A00041FF0E94D678FF91FFBF1F900F90AF91EB
:1059B000BF91CF91DF91EF91FF916F915F914F91E7
:1059C0001895AAEBA4B9AFEFA5B9A0EEA7B9A0E0CE
:1059D000A8B9A0EFAAB9AFEFABB9A6B1AF77A093C2
:1059E0002901B2ECB0938000B9E1B0938100F4E0FA
:1059F000A2FFF4E0F0938700FEEFA2FFF6EFF09332
:105A0000860020928900FAE5F0938800F4E0F09394
:105A10008B00F8EDF0938A00A6E0A0936F00A2E05F
:105A2000A4BDA1E0A5BDA1E3A7BDA3E8A093B000DC
:105A3000A1E0A093B100A0E8A093B3002092B6002B
:105A40002092C000A0E1A093C100A6E6A093C200EE
:105A5000ACE5B0910C01B3FDAFE5ACBDA0E0ADBDD0
:105A6000A5E17AD0C8E0D1E0A8ECA993A1E0A99380
:105A7000AEE12992AA95E9F7AAEAA0931E01A093A4
:105A8000200120922A0120920D01AEE3A0931C0177
:105A90000F93009129010F770093290106EE07C0AB
:105AA0000F930091290100680093290104EE0093EF
:105AB00030010F910895A0933E01A03041F4ACE372
:105AC000A0934401AEE2A0934501A6EE42C0A130EE
:105AD00069F4A8EAA0934401A4E7A0934501A0E0DB
:105AE000A0930001A0EEA093010124C0A23091F484
:105AF000A8E7A0934401ACE4A0934501C0E0D1E045
:105B0000A0E0A993A0E4A993A0EAA993A0EEA99389
:105B1000A3EE1FC0A33081F4A4E5A0934401AAE33F
:105B2000A0934501C0E0D1E0AA27B8E0A993A05E08
:105B3000BA95E1F7A7EE0DC0A0E8A0934401A0E458
:105B4000A0934501A0E2A0930001A0EEA093010163
:105B5000A0ECA09330010895AA0FAE7EA0932C0173
:105B60000895A295AA0FA07EA0930F0108954883DF
:105B70004091290147FD0EC0CF93DF935F9342EB25
:105B8000C40F42E0D41F40912C014E7E48835F91A8
:105B9000DF91CF9108954F935F936F93AF93BF932E
:105BA00040E2592F5370523061F0533009F44BE208
:105BB000B7FF05C0A095B095A30DB21D4DE20E94A0
:105BC000A22E592F5C70692F6073E8944FE24395C1
:105BD000A051B742E0F7A05FB84D5C3009F42BD07C
:105BE0004FE24395A85EB340E0F7A851BC4F53FD88
:105BF00022D0603309F4A3D04FE24395A456B209F2
:105C0000E0F7AC59BF4F503009F015D0603209F4BD
:105C100096D04FE24395AA50E8F70DD0A65F6031C9
:105C200009F48DD040E34A0F8DD0BF91AF916F91B1
:105C30005F914F910895403311F0689483C091FDB6
:105C400081C0F6F390FF08957CC008954F9390FFB4
:105C500005C04B2F429509D04B2F07D04A2F4295B4
:105C600004D04A2F02D04F9108954F70405D4A33BF
:105C700008F0495F67C040913E014030B1F0AF93FA
:105C8000BF93CF93DF93D1E0C8ECACE5BEE129929E
:105C9000BA95E9F7AA95D1F7DF91CF91AA24BB2451
:105CA00020922B01BF91AF910895AF93BF93CF93F3
:105CB000DF93D1E0C8ECA7E1BEE14993BA95E9F7DB
:105CC000AA95D1F740912C014E7EA7E1BEE1499300
:105CD000BA95E9F7AA95D1F7DF91CF91AA24BB2411
:105CE00020922B01BF91AF910895AF93BF93209263
:105CF0002B01A0912A01A03051F4A7E1AA24B3946A
:105D0000AB1571F7B6E1BB2ECF93DF9362C0A13024
:105D100029F4BF91AF914AE00C942B34A23021F4C6
:105D2000BF91AF914AE090C4A33019F4BF91AF91F5
:105D30000895BF91AF915AE00E94263908954CE230
:105D400001C040E2AF93BF93A0912B01A395A09314
:105D50002B01A0912A01A43030F0BF91AF91542FB4
:105D60000E9426390895A030A9F0A33059F4A42F39
:105D7000BB275F936F930E948B176F915F91BF91C9
:105D8000AF910895BF91AF91A0912A01A1FF0C940A
:105D90002B345AC4EF93E0913E01E03009F09AC0F1
:105DA000EF91CF93DF932FD496FD35C0E0DEA3951E
:105DB000AE3131F4AA27B395B73111F4B6E107C07B
:105DC000AA2EBB2EDF91CF91BF91AF910895AA2E3D
:105DD000BB2ED1E0C8EC4F93A6E1BEE14E8D4993B6
:105DE000BA95E1F7AA95C9F7AEE140E24993AA95C1
:105DF000E9F7D4E0CAE7A6E1BEE14E8D4993BA9532
:105E0000E1F7AA95C9F7AEE140912C014993AA9513
:105E1000E9F74F91D7CFAB31A8F6B23198F6AD5F25
:105E2000AA2EEF93FF934F925F926F927F9270F83A
:105E30005F93E42FF6EFB5E04424552466245527FC
:105E4000A491A7FD539550FB40F8A6FD539550FB38
:105E500041F8A5FD539550FB50F8A4FD539550FB18
:105E600051F8A3FD539550FB60F8A2FD539550FBEC
:105E700061F8F3955527A491A7FD539550FB42F87F
:105E8000A6FD539550FB43F8A5FD539550FB52F8E2
:105E9000A4FD539550FB53F8A3FD539550FB62F8B6
:105EA000A2FD539550FB63F8F395442D60DE2196D7
:105EB000452D5DDE2196462D5ADE6C96BA9509F089
:105EC000BBCF5F9170FA7F906F905F904F90FF9182
:105ED000EF9178CFFF93CF93DF936F937F93E42F6E
:105EE00060910D0160FD1EC0F6EFAA2DBB2DDAE01A
:105EF000C49137D0B395AA2D96FD33D096FDB395B6
:105F0000F395AA2DDA95A1F7AA2DAA5F96FDAA5FAF
:105F1000AA2E7F916F91DF91CF91FF91EF91BF9169
:105F2000AF910895FAE7EF77AE2FECEBEA0FF21D91
:105F3000AA0FEA0FF21DAA2DBB2DD6E0C49155D0B1
:105F4000B395AA2D96FD51D096FDB395D0FD31960F
:105F5000AA2DDA9599F7AA2DAC5F96FDAC5FAA2E13
:105F6000D8CF60912C016F936295C7FD62956093C5
:105F70002C01A2D0A39596FD9FD096FDA395C6FDBA
:105F8000629560932C0198D0A39596FD95D096FDCF
:105F9000A395C5FD629560932C018ED0A39596FDC7
:105FA0008BD096FDA395C4FD629560932C0184D09F
:105FB000A39596FD81D096FDA395C3FD6295609350
:105FC0002C017AD0A39596FD77D096FDA395C2FDBE
:105FD000629560932C0170D0A39596FD6DD096FDCF
:105FE000A3956F9160932C01089560912C01D0FDD1
:105FF000C295762FC7FF729570932C015DD0A39543
:1060000096FD5AD096FDA395762FC6FF7295709394
:106010002C0152D0A39596FD4FD096FDA395762FD7
:10602000C5FF729570932C0147D0A39596FD44D07F
:1060300096FDA395762FC4FF729570932C013CD0EA
:10604000A39596FD39D096FDA39560932C010895F4
:106050004F934591403011F44F91089573DEF9CF7D
:10606000FF91EF91EE0FFF1FAF93BF93B591BF3F2D
:1060700011F0A5910ED0BF91AF914F934591403053
:1060800031F44F913197F695E795319609945ADEA0
:10609000F5CFEF93E0913E01E03021F0EF91AA2E91
:1060A000BB2E0895EF91AE3108F0ADE1B73108F0A5
:1060B000B6E1AA2EBB2E0895CF93DF93C091440181
:1060C000CA1728F0C0914501CB1708F003C0DF9133
:1060D000CF910895AF93BF934F935F93C0913E01CB
:1060E000C53021F0C37031F0C23008F441C009F46A
:1060F00064C081C051E0AC3360F5BE3250F5B0FDF4
:10610000550FB0FD550FA0FD550FB695A695CEE1E4
:10611000BC9FD1E0C8ECCA0FD21DC00DD11DA2EBAF
:10612000B2E0CA0FDB1FA881B0912C01BE70B295FE
:10613000A07EBA17A9F0B0912C01BE70AB2BAE7E39
:10614000A883A2EBB2E0CA1BDB0BB881B52BBF70F2
:10615000B8835F914F91BF91AF91DF91CF91089537
:10616000A2EBB2E0CA1BDB0BB8815095B523EFCF91
:10617000CA2FC770C39540E00894441FCA95E9F739
:10618000A695A695A695C5E1D0913E01D2FDC0E1A8
:10619000BC9FD1E0C8ECCA0FD21DC00DD11DA0918B
:1061A0002C01A695A17029F44095A881A423A88369
:1061B000D0CFA881A42BA883CCCFCA2F50912C017B
:1061C0005695537043E0C37031F0440F440F550FA0
:1061D000550FCA95C9F74095A695A695CEE1BC9FE7
:1061E000D1E0C8ECCA0FD21DC00DD11DA881A423D7
:1061F000A52BA883AECFCA2F50912C015E704EE024
:10620000C17011F4429552954095A695CAE2BC9F83
:10621000D1E0C8ECCA0FD21DC00DD11DA881A423A6
:10622000A52BA88396CFCE3108F0CDE1EE3108F052
:10623000EDE1D73108F0D6E1F73108F0F6E1EC17DF
:1062400018F40E2EEC2FC02DFD1718F40F2EFD2F75
:10625000D02D0895EC1718F40E2EEC2FC02DFD173D
:1062600018F40F2EFD2FD02D0895AF93BF93CF9329
:10627000DF93EF93FF935F93D6DFAC2FBD2FCF93C8
:10628000DF93C3D1288252EBC50F52E0D51F509146
:106290002C015883DF91CF91AE1711F0A395EFCF6A
:1062A000BF1719F0AC2FB395EACF5F91FF91EF9133
:1062B000DF91CF91BF91AF910895AF93BF93CF93EB
:1062C000DF93EF93FF935F93C5DFAC2FBD2FF4DE19
:1062D000A395AE17E1F7F0DEB395FB17E1F7ECDE1F
:1062E000AA95AC17E1F7E8DEBA95BD17E1F75F9123
:1062F000FF91EF91DF91CF91BF91AF910895AF934F
:10630000BF93CF93DF93EF93FF935F93A3DFBD2FF3
:10631000AC2FD2DEAE1711F0A395FBCFCDDEFB176D
:1063200011F0B395F5CF5F91FF91EF91DF91CF9190
:10633000BF91AF91089599DFAF93BF93CF93DF9350
:10634000EF93FF934F935F936EDF4C2FBD2FAC2FD6
:106350005CD152EF599351EFA395AE1711F05993B9
:10636000FBCF53EF5993A42FB395BF1739F04DD1FD
:1063700050EF5993AE2F49D15993F5CFA42F45D162
:1063800054EF599351EFA395AE1711F05993FBCFEA
:1063900055EF59935F914F91FF91EF91DF91CF911D
:1063A000BF91AF910895C7DF5F93AF93BF93CF9332
:1063B000DF93EF93FF9337DFBD2FAC2F26D15BEF39
:1063C00059935CEEA395AE1711F05993FBCF5CEF98
:1063D0005993FF91EF91DF91CF91CF93DF93EF939B
:1063E000FF93BD2FAC2FB39510D15DEF599350E2C1
:1063F000A395AE1711F05993FBCF5EEF5993FF9120
:10640000EF91DF91CF91CF93DF93EF93FF93BD2F68
:10641000AC2FB395AF93F9D0A2EBB2E0CA0FDB1F5C
:1064200050912C0152955E7E2196AF91A395AE17A7
:1064300011F05993FBCFFF91EF91DF91CF91CF9363
:10644000DF93EF93FF93BD2FAC2FBE5FDED05EEEE8
:1064500059935DEEA395AE1711F05993FBCF5FEE04
:106460005993FF91EF91DF91CF91BF91AF915F91E0
:1064700008950F931F932F933F93AF93BF93CF93A1
:10648000DF93DE010FEFCE1B10F40195C1951FEFD6
:10649000DF1B10F41195D195CD1760F000C02C2FA3
:1064A00026950ADEAE1789F0A00F2D1BD0F7B10F8D
:1064B0002C0FF7CF2D2F2695FFDDBF1731F0B10F31
:1064C0002C1BD0F7A00F2D0FF7CFDF91CF91BF91ED
:1064D000AF913F912F911F910F910895AF93A82DE8
:1064E000A73EE9F3A82DA73EE9F7AF910895EF93F2
:1064F000FF93AF93A0931D01FBE8A6FDFCE8F0938A
:106500002F01AF73AA0FFDE8E0E8EA0FF21DA59195
:10651000A0931A01A591A0931B0120921C01209227
:10652000180120921901AF91FF91EF9108952092E7
:106530001701409117014030E1F39DC040911601D1
:106540004030E1F708955FD0A2EBCA0FA2E0DA1F56
:10655000A881BA2FAF93A171BE7EB295BA2BAF912D
:106560002092170140911701403041F440911001F1
:106570004B3110F4A883F6CFB883F4CFA8837BD037
:1065800042C03F933DED52D020921701409114013B
:106590004470431749F0403021F40E940F07342F14
:1065A00003C00E943507342F40911701403061F439
:1065B000409110014B3120F448814F774883E6CF5A
:1065C000488140684883E2CF58815F7758833F9184
:1065D0000895D1E0C3EDCA0FD21D2092170140915A
:1065E0001701403061F4409110014B3120F4488193
:1065F0004F774883F4CF488140684883F0CF588173
:106600005F7758830895AA2DBB2DDEE1BD9FD1E0B1
:10661000C8ECCA0FD21DC00DD11D0895F6DF0F932F
:1066200002EBC00F02E0D01F0F910895D3E2BD9F8F
:10663000D2E0C4E3CA0FD21DC00DD11D0895AA2D0A
:10664000BB2DAA95B39525CDBF93B0910C01B4FD98
:106650000EC0BFEFB1B900001A99FECF42B9B4E63F
:10666000BA95F1F72998B4E6BA95F1F7299ABF914E
:1066700008954F9108954F9340912D0141FFF9CF17
:106680004D7F40932D01FF93EF93DF93CF93409184
:106690003E01403029F44091290147FF13C02FC02B
:1066A0004F9347E4D8D04F914F93405DD4D04F9152
:1066B000413009F45AC0423009F470C0433009F443
:1066C0008CC09EC044E50E942B344AE00E942B34CB
:1066D000C8ECD1E0FEE2EEE148814295ADD04991AF
:1066E000ABD0EA95C9F74AE00E942B34FA9599F7A6
:1066F000CF91DF91EF91FF914F914427089545E4A9
:106700000E942B344091400194D04AE00E942B34E7
:10671000C8ECD1E0F3E0E3E2488142958DD04991A5
:106720008BD0EA95C9F74AE00E942B34FA9599F785
:10673000E3E2F0912E01EF9FC00DD11DF0E1E3E205
:1067400048814F77429578D049914F7775D0EA9537
:10675000B9F74AE00E942B34FA9589F7CF91DF917F
:10676000EF91FF914F91442708954091000161D02E
:10677000409101015ED04AE06ED0C8ECD1E0F4E770
:10678000E5E14881429558D0499156D0EA95C9F73C
:106790004AE00E942B34FA9599F7E0CF409100012E
:1067A00048D04091010145D04091020142D0409132
:1067B00003013FD04AE04FD0C8ECD1E0F4E5EEE170
:1067C0004881429539D0499137D0EA95C9F74AE0D6
:1067D0000E942B34FA9599F7C1CF4AE03CD0C8EC1F
:1067E000D1E0FAE3EAE24881429526D0499124D0EB
:1067F000EA95C9F74AE00E942B34FA9599F7AECF93
:106800004091000116D04091010113D04AE023D0FD
:10681000C8ECD1E0F0E4E0E1488142950DD0499127
:106820000BD0EA95C9F74AE00E942B34FA9599F704
:1068300095CF4295469547704F70405D4A3308F0BA
:10684000495F0C942B34BF93B2E0A03009F0B064E0
:10685000B4BDBF910895BF93B0912501B030E1F769
:1068600040932601BA95B0932501BF910895BF9337
:10687000B0912701B030E1F7BA95B0932701B091FC
:106880002701B030E1F740912801BF910895BF93EF
:10689000B0912701B030E1F7BA95B093270140914C
:1068A00016014D3E41F0B0912701B030C1F7409143
:1068B0002801BF9108954BE1BF910895DF93CF93D5
:1068C000BF93AF93FF93EF93CEE0D7E0E4E4F9E614
:1068D00033D0EF91FF91FF93EF93CDDECCE5D4E081
:1068E000B0911401B2FD7E9616F026D001C01ED0E4
:1068F00040911601A1E04D3E69F0A2E0413F51F008
:10690000A3E0423F39F0A4E0433F21F0A5E0443F3B
:1069100009F0DFCFB0911401B2FDAB5F4A2FEF91C8
:10692000FF91AF91BF91CF91DF910895BEE1A19109
:10693000A993BA95E1F70895BEE1A591A993BA95F7
:10694000E1F708954E4E4E4E4E4EC0C0C0C0C0C07E
:106950008080808080802E2E2E2E2E2E6E6E6E6E6B
:106960006E6EACE5B0910C01B3FDAFE5ACBDACE52E
:10697000A093B800A0E0B2FDA1E0A093B9000895F3
:10698000FF93EF930F93E0911E01A0911F01B0912F
:106990002001F09121010027E2FD0095E5FD009521
:1069A000A4FD0095F7FD0095001FEE1FAA1FBB1F59
:1069B000FF1FE0931E01A0931F01B0932001F093ED
:1069C00021010F91EF91FF910895FF93EF93DF93D2
:1069D000CF93BF93AF934F935F936F937F934F92F8
:1069E0005F926F927F922F9320913E0140904601DB
:1069F000509049016090480170904B0150914701BF
:106A000060914A01A22FA370E52F660FEE0FA3300D
:106A100031F0660FEE0FA23011F0660FEE0FF62F79
:106A2000A0914C01A13071F4E20147D0803011F007
:106A30008FE133C0E30141D0803011F080E22DC0FE
:106A400065D02BC0A23091F4E20137D0803011F034
:106A50008FE123C0E30140D0803011F082E11DC0FE
:106A6000ACE3BDE06A0E7B1E75D017C0A33011F0F9
:106A700085E113C0A52DA33010F082E10EC0ACE378
:106A8000BDE04A0E5B1EF20151916191E30115D008
:106A9000803011F080E201C067D02F917F906F901D
:106AA0005F904F907F916F915F914F91AF91BF91A8
:106AB000CF91DF91EF91FF910895CE0F10F48FE108
:106AC0000895A0914401CA17D0F7DF0FC0F3B09129
:106AD0004501DB17A0F70895659FC00DD11D2296D3
:106AE000D33008F082E10895A22F509147016091C0
:106AF0004A01E52F660FEE0FA33031F0660FEE0F5F
:106B0000A23011F0660FEE0FF62F0895571478F0AB
:106B1000D20134D0E0E8FBE064D0D3012FD0E0E82C
:106B2000FBE08CD0539473946A9591F70895560EB8
:106B3000760E5A947A94D20121D0E0E8FBE051D04D
:106B4000D3011CD0E0E8FBE079D05A947A946A959E
:106B500091F70895F30151936193D2010FD041D081
:106B600053946A95D1F70895F20151916191D3013F
:106B700005D064D073946A95D1F708956F93C8ECEB
:106B8000D1E0213011F465E103C0253069F460E102
:106B9000B69FC00DD11D6A2F669566956695C60F86
:106BA000D21D4A2F6F910895223069F46EE1B69F8D
:106BB000C00DD11D6A2F66956695C60FD21D4A2F4E
:106BC000440F6F9108956AE2B69FC00DD11D6A2FE0
:106BD00066956695C60FD21D4A2F440F440F6F91DC
:106BE00008957F936F93BF93AF93652F742F777042
:106BF00049F4A991A1936A95E1F7AF91BF916F9183
:106C00007F910895B0E8713019F0B6957A95FBCF71
:106C10007727A991AB9F703019F0A291A029A19379
:106C2000119273957617A9F7A991AB9FA291A0290C
:106C3000A193AF91BF916F917F9108957F936F93CF
:106C4000BF93AF93652F742F777049F4A191A993E7
:106C50006A95E1F7AF91BF916F917F9108950F937E
:106C60001F930FEF11E0000F110F7A95E1F7652FD9
:106C70007881009570230095A191A19F072A099220
:106C8000712D6A95C9F768816023672B69930F910D
:106C90001F91AF91BF916F917F910895BF93AF9373
:106CA0004F939927A42F0E94262E0E94A12E4F9128
:106CB000AF91BF910895AF93BF93EF93FF935F930D
:106CC0006F930F931F932F9310E020E0FAE8EE27C5
:106CD000509147015F7760914A016F770491059F5A
:106CE000A12DE0950491E095069FB12DA11729F4FF
:106CF000B21719F4E39591F724C01A2F2B2FA09106
:106D00004601B0914901A10FB20F0E945C30A091E1
:106D10004601B0914901A10FB21B0E945C30A091C5
:106D20004601B0914901A11BB21B0E945C30A091A9
:106D30004601B0914901A11BB20F0E945C30E3955E
:106D400069F62F911F910F916F915F91FF91EF91D4
:106D5000DF91AF910895AF93BF93EF93FF935F934C
:106D60006F930F931F932F933F932FEFFAE8EE2724
:106D7000509147015F7760914A016F770491059FB9
:106D8000A12DE0950491E095069FB12DB21721F455
:106D9000E395A1F73F91D5CF1A2F2B2FA091460154
:106DA000B09149013A2FB21BA11B310F0E945C30F8
:106DB000B20FB20F0E945C30B21BB21BA3953A1700
:106DC000A8F7E395D9F63F91BCCFFF91EF91EE0F75
:106DD000FF1F5BD03197F695E7953196EF93FF93C0
:106DE000C8E7D1E040912C014F93FF93EF9361D01E
:106DF0000E9430300B0920505245535320454E54C9
:106E000045522000EF91FF914F9140932C018FDB71
:106E10004A3EE9F793DB0E94E5190895FF91EF914F
:106E2000EE0FFF1F32D03197F695E7953196EF932D
:106E3000FF93C8E7D1E040912C014F93FF93EF936C
:106E400038D00E9430300B08202859296573202F34
:106E500020284E296F200000EF91FF914F91409321
:106E60002C0165DB493761F0493551F04E3619F098
:106E70004E3409F0F6CF62DB0E94E51944270895ED
:106E80005DDB0E94E51941E00895C8E7D1E0459136
:106E900046954F93477049934F9142954770499358
:106EA00058E145914993403011F05A95D1F7299214
:106EB0000895FF93EF9392E020922A01A991B9914E
:106EC000B295B077A770AB0FAA0FA0932C01DF93F8
:106ED000CF930E94BF19C2E0D8E0EBE1FCE00E9432
:106EE0009B31A3E0B9E00E944930CF91DF9158E196
:106EF0004991403051F0DF93CF935F930E94A22ECF
:106F00005F91CF91DF915A9599F740912C0142956D
:106F100040932C01EF91FF910895FF93EF93DF933E
:106F2000CF93BF93AF93C0914601D09149010A819D
:106F300019810E3118F4173108F41AD0A0914801C4
:106F4000B0914B01C0914601D0914901B983AA8308
:106F5000AE3138F4B73128F43DD07370713009F098
:106F600076D0AF91BF91CF91DF91EF91FF910895CE
:106F7000C0914601D09149010A8119812C813B8140
:106F8000239F310F2596C00DD11DC00DD11D412F5E
:106F9000E8ECF1E05EE1549FE00DF11DE00FF21D21
:106FA000522F699161935A95E1F74395431781F701
:106FB000412FEAE7F4E05EE1549FE00DF11DE00FA0
:106FC000F21D522F699161935A95E1F7439543174A
:106FD00081F70895C0914601D09149010A81198134
:106FE0002C813B81239F310F2596C00DD11DC00DF3
:106FF000D11D7727412FE8ECF1E05EE1549FE00DD1
:10700000F11DE00FF21D522F619169936F7009F02D
:1070100071E05A95C9F74395431769F7E091460126
:10702000F09149014081742B7083412FEAE7F4E02D
:107030005EE1549FE00DF11DE00FF21D522F6191B2
:1070400069935A95E1F74395431781F70895C091E5
:107050004601D09149010A8119812C813B81310F70
:107060002596412FE8ECF1E05EE1549FE00DF11D23
:10707000E00FF21D522F699161935A95E1F7439504
:10708000431781F7412FEAE7F4E05EE1549FE00DFA
:10709000F11DE00FF21D522F6991660F28F46E70FA
:1070A000462E6081607F642961935A95A9F74395C4
:1070B000431749F70895AF93BF93CF93DF934F934F
:1070C0005F936F937F934F9270912C014370E1F423
:1070D000A6E0B2E0C4E2D2E0422C07D0A8EBB4E0D4
:1070E000C6EDD4E0472E01D061C062E15AE149917A
:1070F0004D935A95E1F7149624966A95B9F75AE19B
:107100004D925A95E9F708954130C9F4ACE3B4E0E3
:10711000CBE3D4E0422C07D0AEEEB6E0CDEED6E025
:10712000472E01D043C063E159E14A914E935A95ED
:10713000E1F74E92149725976A95B1F7089542307A
:10714000E1F4ACE3B4E0CEE1D4E0422C07D0AEEE03
:10715000B6E0C0EDD6E0472E01D028C062E15AE18A
:107160004A914E935A95E1F7149724976A95B9F787
:107170005AE14E925A95E9F70895A6E0B2E0C7E0C9
:10718000D2E0422C07D0A8EBB4E0C9EBD4E0472E04
:1071900001D00CC063E159E149914D935A95E1F753
:1071A0004D92259614966A95B1F708954F907F9168
:1071B0006F915F914F91DF91CF91BF91AF91089502
:1071C0004F935F937F9363DB4B3111F481E015C0E4
:1071D0004130C9F74CDB642F4ADB4095641711F04E
:1071E00088E20BC070E8552742DB540F49937A952B
:1071F000D9F73DDB451729F488277F915F914F919F
:10720000089589E2FACF4F935F937F9341E023DBA8
:10721000462F21DB40951FDB70E855274991540F1D
:107220001ADB7A95D9F7452F16DB7F915F914F9145
:1072300008955E984CE54093B80044E84093BC0044
:1072400044E94093BC00089544EA0EC05093BB004B
:1072500044E80AC044EC08D05091BB00089544E8CB
:1072600003D05091BB0008954093BC004091BC00F6
:1072700047FFFCCF6091B900687F0895E5DF683073
:1072800089F4572F550F5E70506AE0DF683151F472
:107290005B2FDCDF683231F45A2FD8DF683211F40B
:1072A000882708958FE0CCCFCFDF6031D9F7572FF3
:1072B000550F5E70516ACADF6034A1F788270895C0
:1072C000DDDF803049F4F0DF803031F4C8DF68352D
:1072D00019F411968827B4CF8FE0B2CF5F93CEDF39
:1072E0005F91803031F4B2DF683219F4119688274B
:1072F000A7CF8FE0A5CFA8DF6830A9F4572F57702C
:10730000550F5169A3DF603471F4A4DF603559F47F
:10731000A52FA5DF683539F4BB27550FAA1F08F440
:10732000B09588278DCF8FE08BCF8827D83020F07D
:1073300080E34F914F914FEF0895F7DFF999FECF1A
:10734000D2BDC1BDF89A40B521960895EEDFF999F6
:10735000FECFD2BDC1BDF89A40B4441611F42196B7
:10736000089554E040BDF894FA9AF99A7894F999FE
:10737000FECFF89A40B4441511F4219608958395F0
:1073800080635A9579F70895AF93D7DF4193AA9513
:10739000E1F7AF910895AF934191D8DFAA95E1F756
:1073A000AF9108954EBD4DB547FFFDCF4EB5089541
:1073B00088272C9847EDF6DF4427F4DF2C9A4C7B86
:1073C0004432B1F34C31A1F38827443A19F04C39D7
:1073D00009F081E108958827EBDF803021F040E05B
:1073E00040939C1008954C3911F448E0F9CF40E1E6
:1073F000F7CFF1DF403009F40895440F440F440FF4
:10740000440F4A950895AA0FBB1F4B2FCBDF4A2F7D
:10741000C9DF422DC7DFB695A7950895803059F48E
:107420004F93C6DF803031F42C9845E5BBDFEBDFAE
:107430002C9ABEDF4F910895803059F44F93B8DFF6
:10744000803031F42C9843E5ADDFDDDF2C9AB0DFDE
:107450004F910895803051F44F93AADF803029F482
:107460002C9846E89FDFCFDF2C9A4F910895119614
:10747000B0939D10A0939E101197ECCF7F93772728
:1074800010D07F9108957F9371E00BD0D42F72E0DC
:1074900008D0C42F7F9108957F9373E002D07F912D
:1074A00008958030B9F484DF8030A1F42C9842ED47
:1074B00079DFAA0FBB1FA3954B2F74DF4A2F72DF12
:1074C000472F70DFB695A7956DDF6CDF6BDF6ADF46
:1074D00069DF2C9A08958030D1F46ADF8030B9F4E6
:1074E0002C9842ED5FDFAA0FBB1F4B2F5BDF4A2FAB
:1074F00059DF472F440F56DFB695A79553DF52DF6C
:1075000051DF50DF4FDFD42F4DDFC42F2C9A089569
:107510007F9370E010D07F9108957F9371E04D2F9D
:107520000AD072E04C2FBDDF7F9108957F9373E006
:10753000B8DF7F9108958030A1F44F9339DF4F91E8
:10754000803079F42C984F9347E82CDF44272ADFCA
:1075500041E028DF472F26DF4F914F9323DF2C9AFE
:107560004F910895803091F423DF8030D1F72C982B
:107570004F9347E817DF442715DF40E013DF472F1D
:1075800011DF4F914F930EDF2C9A4F910895803069
:10759000D1F4DF93CF934F935F930ADF803079F478
:1075A0002C9847E8FFDE4427FDDE4427FBDE40E061
:1075B000F9DE55274991F6DE5A95E1F72C9A5F914D
:1075C0004F91CF91DF9108958030B1F44F935F9345
:1075D000EFDE803079F42C9847E8E4DE4427E2DEE1
:1075E0004427E0DE40E0DEDE55274FEFDBDE5A9534
:1075F000E1F72C9A5F914F9108958030E1F4DF9389
:10760000CF934F935F93D4DE803089F42C9846ED6E
:10761000C9DE4427C7DE4427C5DE40E0C3DE442779
:10762000C1DE5527BFDE49935A95E1F72C9A5F9149
:107630004F91CF91DF910895BF93AF93DF93CF9395
:107640004F935F937F93C7DE403041F47F915F910A
:107650004F91CF91DF91AF91BF910895B5DF4FE08A
:1076600057DF442763DFAA27BB27F4DE11964DEFCF
:10767000CA2FCF70C13009F44CEF4ADF442756DFE0
:10768000CC27DD274ADFE6DE1196A03019F445EE5F
:107690000E94A22E40919C10B41749F7D7CFBF93F8
:1076A000AF93DF93CF934F935F937F9394DE4030FC
:1076B00091F47F915F914F91CF91DF91AF91BF9105
:1076C0000895B42FAA271197E7DEC42FBB27AA2756
:1076D000E3DE4C1731F4A2DEDFDE439527DFBADEAE
:1076E000E8CF1196D9DE4C17E1F7F5CFDF93CF93B2
:1076F0004F9394DE4DEFCA2FCF70C13009F44CEF99
:1077000007DFC1DE219609DF5FDFA4DE4F91CF9155
:10771000DF910895FF93DF93CF93BF93AF93AA2791
:10772000BB27ED0158DE4030A1F0F42FA7DE4C3F1F
:1077300041F04D3F31F04B3A21F04F3018F04039D5
:1077400008F421961196BF1789F74427DF1709F42B
:1077500041E0AF91BF91CF91DF91FF9108950F93D9
:10776000BF93AF934F93AA27BB27ED01FD0133DEF3
:10777000403099F0042F82DE4D3F49F4DF93CF93E0
:1077800082DE4D2FCF91DF914F3F21F021964C3F6C
:1077900009F431961196B01771F74F91AF91BF91DF
:1077A0000F910895FF93EF93DF93CF934F932F9310
:1077B00012DE4030A9F0AA27BB2760DE242FB0914B
:1077C0009D10A0919E1040910801B41710F0A2E006
:1077D000BB27FD0153DE4D3F51F455DED21738F47F
:1077E0002F914F91CF91DF91EF91FF9108951596D1
:1077F00040919C10B41709F4BB27BF1759F7AE1777
:1078000049F7AA27BB270ADE39DE4F3F31F0405F38
:10781000242F7EDE1FDEDF01DDCFAFEFBFEFE0CF35
:10782000FF93EF93DF93CF93BF93AF934F935F9308
:107830006F937F93D0DD403061F481E17F916F9150
:107840005F914F91AF91BF91CF91DF91EF91FF91F8
:10785000089551D0B41710F08BE1F0CF0FDE4C3FFC
:1078600011F087E1EBCF40915A01403011F48BE1E8
:10787000E5CF413810F08BE1E1CF71DFD03021F45A
:10788000C41710F488E1DACFC0E8DBE050E06FEF16
:1078900069935A95E9F798DE1196B0939D10A093DD
:1078A0009E1040915A01C0E8DBE04F937BDFB99313
:1078B000A9934BEA2DDEDF93CF93E5DD21962DDEF4
:1078C000CF91DF91E9DD32DED2DDE9DE4F914A95DD
:1078D00061F711D0C0E8DBE05ADE40915C0118DEB0
:1078E000DF93CF93D0DD219618DECF91DF91D4DDE9
:1078F0001DDEB0DDA3CFA0915801A295BA2FA07FC5
:10790000BF7011960895BF93AF93DF93CF934F93BA
:107910005F937F937727EFDFB1DD4C3F69F0DBDDCD
:10792000DF3F49F0BF93AF93DE01E0DEAF91BF913F
:10793000B6DE7F5FA1F7DADE7F915F914F91CF9145
:10794000DF91AF91BF910895BF93AF93DF93CF9332
:107950004F935F937F932F93AA27BB2729DD8EDD5B
:10796000242FC9DF8BDD4C3F51F489E12F917F91AA
:107970005F914F91CF91DF91AF91BF910895709139
:107980005A01703810F08BE1F1CFA5DDDF3F11F423
:107990008BE1ECCFDE01CCE3DDE040915C014130D6
:1079A00009F4D395423009F4DE5FF1DDDF93CF9324
:1079B0006ADDD21759F02196B0DDCF91DF915EDDFF
:1079C000A7DD6ADDB3DD46DD6ADED0CF8FDEEADE1D
:1079D0005ADD2196A2DDCF91DF914BEA99DD5CDD86
:1079E000A5DD38DDED0187DF19DD70915A01770FD4
:1079F0004D2FB8DD73954C2FB5DD40DD89DD4CDDB5
:107A000095DD28DDB3CFBF93AF93DF93CF934F9333
:107A10005F937F9370DF32DD4C3F49F48EE17F91BD
:107A20005F914F91CF91DF91AF91BF910895709188
:107A30005A01703810F08BE1F2CF4DDDDF3F11F4C9
:107A40008BE1EDCFDE01EADCCCE3DDE040915C01CF
:107A5000413009F4D395423009F4DE5FCEDDDFCF4B
:107A60000004080D11161A1F23282C3035393D4209
:107A7000464A4F53575B5F64686C7074787C7F83B1
:107A8000878B8F92969A9DA1A4A7ABAEB1B5B8BBD8
:107A9000BEC1C4C6C9CCCFD1D4D6D9DBDDDFE2E4C8
:107AA000E6E8E9EBEDEEF0F2F3F4F6F7F8F9FAFBBD
:107AB000FCFCFDFEFEFFFFFFFFFFFFFF000000CC10
:107AC000C000333000FFF000000CCCCCCCCC333CF9
:107AD000CCFFFCCC000333CCC333333333FFF3335D
:107AE000000FFFCCCFFF333FFFFFFFFFA5A5A5068B
:107AF000FF60000000000000000000000000000027
:107B00000000000000000000000000000000000075
:107B10000EAE000004E000AAE800EE4E00000044B3
:107B20004040AA000066FF666842C4A248A0000068
:107B3000004400004888404222400A4A0004E40011
:107B400000048000E000000040224880EAAAE04CE7
:107B500044E0E2E8E0E2E2E0AAE220E8E2E0E8EA8B
:107B6000E0E24880EAEAE0EAE2E00404000404809B
:107B70002484200E0E00842480C268E400EEE04AD3
:107B8000AEA0CACAC0688860CAAAC0E8C8E0E8C88F
:107B90008068EA60AAEAA0E444E0E22A60AC8CA033
:107BA0008888E0AEAAA0CAAAA04AAA40EAE8804A09
:107BB000AA60EAECA068E2C0E44440AAAAE0AAAA4B
:107BC00040AAAEA0AA4AA0AA4440E248E0644460A9
:107BD00004A400C444C04A00000000E04400004A7D
:107BE000AEA0CACAC0688860CAAAC0E8C8E0E8C82F
:107BF0008068EA60AAEAA0E444E0E22A60AC8CA0D3
:107C00008888E0AEAAA0CAAAA04AAA40EAE8804AA8
:107C1000AA60EAECA068E2C0E44440AAAAE0AAAAEA
:107C200040AAAEA0AA4AA0AA4440E248E024C42048
:0C7C30004444448464808842208CEC8032
:1086000000F900F5F3F1F2FC00FAF8F6F4EB5E0085
:10861000F7000000007131000000797361773200CB
:108620000063786465343300002076667472350028
:10863000006E6268677A360000006D6A7537380030
:10864000002C6B696F303900002E2D6C00707E009D
:1086500000000000002700000000EA2B00230000BB
:10866000003C00000000EC00003100343700000046
:10867000302C32353638ED00FB2B332D2A390000F3
:1086800000F900F5F3F1F2FC00FAF8F6F4EB000063
:10869000F70000000051210000005953415722000B
:1086A00000435844452440000020564654522500BB
:1086B000004E4248475A260000004D4A552F2800D8
:1086C000003B4B494F3D2900003A5F4C00503F00B2
:1086D00000000000006000000000EA2A00270000FF
:1086E000003E00000000EC000031003437000000C4
:1086F00030E932353638ED00FB2B332D2A390000B6
:108700000000000000000000000000000000000069
:108710000000000000000000000000000000000059
:108720000000000000000000000000000000000049
:1087300000000000000000C000000000000000C1B8
:10874000000000000000000000002F0000000000FA
:1087500000000000000000000000EA000000C2006D
:10876000000000000000000000E100E2E000000066
:10877000E8E9E500E3E4ED00FB2BE72D2AE6000045
:1087800000000000000000000000000000000000E9
:108790000000000000400000000000000000000099
:1087A00000000000000000000000000000000000C9
:1087B000000000000000000000000000007B5B00E3
:1087C00000000000007D5D000000000000007E0051
:1087D00000000000000000000000005C000000003D
:1087E000007C00000000000000E100E2E00000006A
:1087F000EFEEE500E3E4ED00FB2BE72D2AE60000B9
:1088000000F900F5F3F1F2FC00FAF8F6F4EB5E0083
:10881000F70000000071310000007A7361773200C8
:108820000063786465343300002076667472350026
:10883000006E62686779360000006D6A753738002F
:10884000002C6B696F303900002E2F6C3B702D00AF
:10885000000027005B3D00000000EA5D007E000094
:10886000000000000000EC00003100343700000080
:10887000302C32353638ED00FB2B332D2A390000F1
:1088800000F900F5F3F1F2FC00FAF8F6F4EB000061
:10889000F70000000051210000005A5341574000EA
:1088A00000435844452423000020564654522500D6
:1088B000004E424847595E0000004D4A55262A00A6
:1088C000003C4B494F292800003E3F4C3A505F0086
:1088D000000022007B2B00000000EA7D007C0000ED
:1088E000000000000000EC00003100343700000000
:1088F00030E932353638ED00FB2B332D2A390000B4
:108900000000000000000000000000000000000067
:108910000000000000000000000000000000000057
:108920000000000000000000000000000000000047
:1089300000000000000000C000000000000000C1B6
:10894000000000000000000000002F0000000000F8
:1089500000000000000000000000EA000000C2006B
:10896000000000000000000000E100E2E000000064
:10897000E8E9E500E3E4ED00FB2BE72D2AE6000043
:1089800000000000000000000000000000000000E7
:1089900000000000000000000000000000000000D7
:1089A00000000000000000000000000000000000C7
:1089B00000000000000000000000000000000000B7
:1089C00000000000000000000000000000000000A7
:1089D0000000000000000000000000000000000097
:1089E000000000000000000000E100E2E0000000E4
:1089F000E8E9E500E3E4ED00FB2BE72D2AE60000C3
:108A0000FFFFFFFFFFFFFFFFFFFFFFFEFEFEFEFE7B
:108A1000FEFEFDFDFDFDFDFCFCFCFCFBFBFBFBFA93
:108A2000FAFAF9F9F9F8F8F8F7F7F6F6F6F5F5F4D1
:108A3000F4F3F3F2F2F2F1F0F0EFEFEEEEEDEDEC35
:108A4000EBEBEAEAE9E8E8E7E6E6E5E4E4E3E2E1BD
:108A5000E1E0DFDEDEDDDCDBDADAD9D8D7D6D5D46B
:108A6000D4D3D2D1D0CFCECDCCCBCAC9C9C8C7C63A
:108A7000C5C4C3C2C1BFBEBDBCBBBAB9B8B7B6B529
:108A8000B4B2B1B0AFAEADACAAA9A8A7A6A5A3A237
:108A9000A1A09E9D9C9B99989796949392918F8E5E
:108AA0008D8B8A898786858382817F7E7D7B7A789C
:108AB0007776747371706F6D6C6A696766656362EF
:108AC000605F5D5C5A595756545351504E4D4B4A56
:108AD0004847454442413F3E3C3B393836353332C6
:108AE000302E2D2B2A2827252422201F1D1C1A1941
:108AF00017161412110F0E0C0B09070604030100C0
:108B00000C11161A1E2225282B2D2F313233333407
:108B100034343434343434343535363738393B3CF6
:108B20003E40434547494B4D4F5152535454545482
:108B3000545351504E4C4A4745423F3D3A383634E3
:108B40003231302F2E2E2E2F303132333536383A07
:108B50003C3E4042444647494A4B4D4E4E4F505092
:108B60005050505050504F4E4D4C4B494846434149
:108B70003E3B37332F2B27221D18130D0802FDF81B
:108B8000F3EEE9E5E1DDDAD7D4D2D0CECDCCCCCB53
:108B9000CBCBCBCBCBCBCBCBCACAC9C8C7C6C4C344
:108BA000C1BFBCBAB8B6B4B2B0AEADACABABABAB98
:108BB000ABACAEAFB1B3B5B8BABDC0C2C5C7C9CB17
:108BC000CDCECFD0D1D1D1D0CFCECDCCCAC9C7C5D3
:108BD000C3C1BFBDBBB9B8B6B5B4B2B1B1B0AFAF28
:108BE000AFAFAFAFAFAFB0B1B2B3B4B6B7B9BCBE51
:108BF000C1C4C8CCD0D4D8DDE2E7ECF2F7FD02075F
:108C0000000A141D272F383F464B505457595959C5
:108C1000585654504C48433E39332E2925201C19B0
:108C200016141211111112131517191C1F222527C2
:108C30002A2C2E303132323232312F2D2B28252260
:108C40001F1C191613110F0D0C0B0A0A0A0B0C0E20
:108C500010121416181A1C1E1F2020201F1E1C196B
:108C600016120D0803FDF7F0EAE3DDD6D1CBC6C23C
:108C7000BFBDBBBABBBCBEC2C6CBD1D7DFE6EFF728
:108C80000008101920282E34393D41434445444200
:108C9000403D39342E29221C150F0802FCF7F2ED55
:108CA000E9E6E3E1E0DFDFDFE0E1E3E5E7E9EBED83
:108CB000EFF1F3F4F5F5F5F4F3F2F0EEECE9E6E3B9
:108CC000E0DDDAD7D4D2D0CECDCDCDCDCECFD1D37D
:108CD000D5D8DADDE0E3E6E8EAECEDEEEEEEEDEB3A
:108CE000E9E6E3DFDAD6D1CCC6C1BCB7B3AFABA9F6
:108CF000A7A6A6A6A8ABAFB4B9C0C7D0D8E2EBF57B
:108D000080675342352B221C16120E0C09070605EC
:108D1000040000000000000000000000000000004F
:108D20000000000000000000000000000000000043
:108D30000000000000000000000000000000000033
:108D40000000000000000000000000000000000023
:108D50000000000000000000000000000000000013
:108D60000000000000000000000000000000000003
:108D700000000000000000000000000000000000F3
:108D8000890091009A00A300AD00B700C200CE0098
:108D9000DA00E700F4000301120123013401460167
:108DA0005A016E0184019B01B301CD01E901060264
:108DB0002502450268028C02B302DC020803360376
:108DC00067039B03D2030C0449048B04D0041905E8
:108DD0006705B90510066C06CE063507A307170808
:108DE000930815099F09320ACD0A720B200CD80C82
:108DF0009C0D6B0E460F2F1025112A123F13641481
:108E0000F894A0E02A2EA1E03A2EA0E1AEBFAFEF89
:108E1000ADBFB0E0A0E0AA95F1F7BA95D9F7AAEBFB
:108E2000A4B9AFEFA5B9A0E8A7B9A0E0A8B9A0EF91
:108E3000AAB9AFEFABB9A6B1AF71A09329014B9915
:108E40005DC0B2ECB0938000B9E1B0938100F4E072
:108E5000A2FFF4E0F0938700FEEFA2FFF6EFF0939D
:108E6000860020928900FAE5F0938800A2E0A093A2
:108E70006F00A0E4A4BDA1E0A5BDA1E3A7BD209221
:108E8000C000A0E1A093C100A6E6A093C200E0EA62
:108E9000FFE87ED0A2E2B591B993AA95E1F705B7B4
:108EA000036005BF0E7F05BF7894A8EC68D0B09131
:108EB000C600B83719F0AA95C9F720C0E0ECFFE862
:108EC00067D045E140D0C8ECD1E020D046E03BD0AF
:108ED000E0E0F0E0CCE3DFE019D046E034D0CCEBCA
:108EE000DFE014D0FE3820F40E947A79329678942C
:108EF00046E029D0AEEDB1E01BD0ECCFF89405B739
:108F0000016005BF0C7F05BF0C94000028D04430E1
:108F100039F446E018D0B0912501B030E1F7EECF3A
:108F200050E81DD01CD01BD049935A95E1F717C0CB
:108F30004F2F429501D04F2F4F70405D4A3308F0BC
:108F4000495F4D930895BF93B0912501B030E1F78B
:108F500040932601BA95B0932501BF910895BF9320
:108F6000B0912701B030E1F7BA95B0932701B091E5
:108F70002701B030E1F740912801BF910895AF93E8
:108F8000A82DA73EE9F3A82DA73EE9F7AF910895D4
:108F9000C8ECD1E0A2E2B591B993AA95E1F70895A2
:108FA0004156522D436869704261736963322028CB
:108FB0004631313D557064617465205379732920C1
:108FC000426F6F746C6F61646572204572726F726C
:108FD000202845534320746F206578697429202028
:0E900000202020202020202020202020FF00E3
:0E9C0000202020202020202020202020FF00D7
:0EA80000202020202020202020202020FF00CB
:0EB40000202020202020202020202020FF00BF
:0EC00000202020202020202020202020FF00B3
:0ECC0000202020202020202020202020FF00A7
:0ED80000202020202020202020202020FF009B
:0EE40000202020202020202020202020FF008F
:10F000000C94004700000000000000000000000019
:10F0100000000000000000000000000000000000F0
:10F0200000000000000000000000000000000000E0
:10F03000000000000C941C784F935F936F93FF9334
:10F04000EF93DF93CF93BF93AF930F921F92FFB7CE
:10F05000FF93C8E0D1E0B9A5B7FF5C98B7FD5C9A13
:10F060004B99BE7F4B9BB160B9A7830C921CE9A161
:10F07000F92DF03029F4F82DFA3010F1F63EF8F0C1
:10F08000FCE0E2FFFDEE8F1639F45E98E3FF17C057
:10F09000B2E8B093800013C0F1E1E2FFF3EF8F1606
:10F0A00039F45E9AE3FF0BC0B2ECB093800007C066
:10F0B000F9E3E2FFF7E08F1611F4882499242CC0BD
:10F0C000A0918400AA3FE0F3AB3F00F0AC3F00F01A
:10F0D000AD3F00F0AE3F00F0A8ECB1E0F6EFF80D68
:10F0E000C0E2ED91549140E060E848B9ED9156FDE1
:10F0F00066B90000000055FD66B9049054FD66B97C
:10F10000CA95000053FD66B90000000052FD66B9C3
:10F11000502D59F7000028B814D0E091C600E6370A
:10F1200011F40C947E47FF91FFBF1F900F90AF9199
:10F13000BF91CF91DF91EF91FF916F915F914F91CF
:10F140001895A0913101E0912701E03091F0EF3F57
:10F1500021F4A0FD0EC0EEE30CC0EA95F5EFB491EA
:10F16000B5FF07C0B0912801B695A0FBB7F9B093E1
:10F170002801E0932701E0912501E03091F0EF3F75
:10F1800019F4E8E4AF770DC0EA95F5EFB491B4FF58
:10F1900008C0B0912601B0FB0894B795A7F9B093C9
:10F1A0002601E0932501A09331010895A09131013A
:10F1B000E0912701E03091F0EF3F21F4A0FD0EC077
:10F1C000ECE70CC0EA95F5EFB491B7FF07C0B0913A
:10F1D0002801B695A0FBB7F9B0932801E093270169
:10F1E000E0912501E030E9F2EF3F19F4E0E9AF7773
:10F1F000D8CFEA95F5EFB491B6FFD3CFB091260101
:10F20000B0FB0894B795A7F9B0932601CACF4091F7
:10F210000C01C8EFD7E00E94A6390895C8EFD7E0E7
:10F220000E949D3940930C010895C9EFD7E00E94D8
:10F23000A6390895CF93DF93C9EFD7E00E949D3997
:10F24000742FDF91CF910895FF93EF93DF93CF93C6
:10F25000AF93F4D0E0933401F0933501AF91CF91A7
:10F26000DF91EF91FF910895E0E0F0E9C0E0DCE08C
:10F27000A42FA03021F0EC0FFD1FAA95FACF08951E
:10F28000E0913401F0913501A0E2A99FE00DF11D5C
:10F29000B096C0EAD1E0A0E2B591B993AA95E1F7A2
:10F2A000BFEFB993089547B740FDFDCFB7BFE895CD
:10F2B00047B740FDFDCF089547B746FF0895B1E138
:10F2C000F2DFFACFF8944E2F407E19F4B3E0EBDF73
:10F2D000F3DFA0E109901990B1E0E5DF3296AA953D
:10F2E000C9F7E03009F008953297B5E0DCDFE4DFDC
:10F2F00032960895F8944F93BF93AF93B3E0D3DF62
:10F30000DBDF3297CCE3DFE0A0E83296099019907A
:10F31000B1E0C9DFAA95C9F7B5E0C5DFCDDFAF9190
:10F32000BF914F910895E0913401F0913501B0976C
:10F33000ACE0B591B993AA95E1F7A0912901A7FD99
:10F340000895A6EAB2E0CA0FDB1FACE0B0912C0131
:10F35000B993AA95E9F70895E0E0F0E9A0E0BCE0F0
:10F36000492F403029F3EA0FFB1F4A95FACFF89452
:10F3700063D0C0EAD1E0A3EDB1E05CE04D914993E8
:10F380005A95E1F742E4499353E140E2B9935A9523
:10F39000E9F7A09797DF9927B3E2B99FA4E3B2E01A
:10F3A000A00DB11DC8E7D1E050E24D9149935A95A7
:10F3B000E1F7299250E24A91403219F428825A9595
:10F3C000D1F70E942718C0EAD1E07CDF93959F35E2
:10F3D00019F77894089530D0A3EDB1E05CE0459141
:10F3E0004D935A95E1F77496992750E2A0EAB1E05F
:10F3F00045914D935A95E1F7A8E7B1E040E253E219
:10F400004D935A95E9F7FF93EF939F930E9411193B
:10F410009F91EF91FF91C8E7D1E0B3E2B99FA1E3DB
:10F42000B2E0A00DB11D53E249914D935A95E1F719
:10F4300093959F35D1F6089540913D01AF93BF93C9
:10F44000E0E0F0E947704295A0ECA49FE00DF11DCB
:10F45000BF91AF910895CCE3DFE04CE050E25993C7
:10F460004A95E9F75FEF599343E150E259934A9582
:10F47000E9F740EF5FEF59934A95E9F7DDDF3ADFAF
:10F480003296CCE3DFE040E25FEF59934A95E9F72B
:10F490004BE04F932FDF32964F914A95D1F77894F6
:10F4A0000895472F4770CADFFF93EF93C5DFAF91F1
:10F4B000BF914CE04F93CCE3DFE040E0559159938E
:10F4C0004A95E1F7FF93EF93FD0114DF3296DF01D8
:0EF4D000EF91FF914F914A9569F77894089556
:10F50000010101010101210101010101013181011B
:10F510000100003100010101010131C101010101BE
:10F520003101010101010131C1010101013101017B
:10F530000101010131C101010101110101010101BB
:10F540000111C1010101010101010101010101C11B
:10F55000010101010101010101000101C1010101DC
:10F56000010101010101010001C1010101010100CD
:10F57000010101010101410001010101010101003D
:10F58000000000400000000000000000000000003B
:10F59000000000000000000000000000000000006B
:10F5A000000000000000000000000000000000005B
:10F5B000000000000000000000000000000000004B
:10F5C000000000000000000000000000000000003B
:10F5D000000000000000000000000000000000002B
:10F5E000100000000000000000000000000000000B
:10F5F00020000000000000000000000000000000EB
:10F60000009010800090108000901080009010807A
:10F61000FC28288004C0145028282800000000007E
:10F6200000000000000000000000000000000000DA
:10F6300000000000000000000000000000000000CA
:10F6400000000000000000000000000000000000BA
:10F6500000000000000000000000000000000000AA
:10F66000000000000000000000000000000000009A
:10F67000000000000000000000000000000000008A
:10F6800028C004C00000000000000000000000804E
:10F69000C0A0888400000000000000002088FCB4A6
:10F6A0000028000008A08080000004C028800024FA
:10F6B00000008000000044288000C004C41800003E
:10F6C000000000000000000000000000C004000076
:10F6D0008090808008A084408080C8A400004C8472
:10F6E0000000000000000000C00480800080282886
:10F6F000280000002828002828282800002CE8904E
:10F700000090108000901080009010800090108079
:10F710007C444480A8A814504844440024000000BD
:10F7200000183C3C185028280C3000000000000055
:10F73000241824400C401440242400000C003024E1
:10F7400024244424444040246424106460646424D9
:10F7500044244424406464646464404800481800BD
:10F76000300060000400140060180C6028000000E5
:10F7700000000000300000000000000C18306000A5
:10F7800028A004C0808044283C3C3C000044A88061
:10F79000C0A08884000000000000008040847C58E5
:10F7A000182800001090808004C004C028FC287C29
:10F7B00000440C00000044EC8000C004C42400009D
:10F7C000000000000000000000008080C004000075
:10F7D0008088A41010908440C004C8A400008C80CD
:10F7E000287C008080004084FCF4C0040000244891
:10F7F000280000002828002828282800002CE8C01D
:10F800000090108000901080009010800090108078
:10F81000FC44448080801450444444283C00000050
:10F8200000183C3C20546C181818181800000004EC
:10F830006428640C14603064646428281800186418
:10F84000646464646460606464180C6C605864642C
:10F8500064646464186464646464046000183C0054
:10F860001800600004003400600000601800000010
:10F870000000000030000000000000181818601898
:10F88000449008A0C4C4806C0000001C1844A880E8
:10F89000C0A0888400000000000080804084FCB488
:10F8A0002428282820888080A4A00C60448044401C
:10F8B00000440C40844444800000C0046C24004494
:10F8C00000000000000000000000C004C004481058
:10F8D0008084BCB020888820D834C8A440848C8020
:10F8E0002C7C00C4C444C004E094C0040080208880
:10F8F000280000002828002828282800002CE8A03C
:10F900000090108000901080009010800090108077
:10F910007C808080808010908480804424186424BF
:10F9200000183C40780C7830300C7C180000000C3B
:10F93000681804183C44600C6464282830400C04A7
:10F94000046464606460606064180C78607C546473
:10F9500064646460186464643C640C60301864001F
:10F960000C2444242C2430207428146C185C742437
:10F970004824742448646464646440181818300C83
:10F9800044881090C4BC446C24246434286C6C807B
:10F99000C0A08884000000000080808080807CEC13
:10F9A000404444442088408490A00C6044FC286477
:10F9B00000440C40844444280000C0046C240080AF
:10F9C00000000000000000000000C004C00418187F
:10F9D0008080BC1040848820E82CC8A480804C849F
:10F9E000EC2400C4EC44C004E094C00400802088EF
:10F9F000280000002828002828282800002CE8E4F7
:10FA00000090108000901080009010800090108076
:10FA1000FC808080B098109080ECEC44003C6464E2
:10FA20000018003C24183000300C2440004000181E
:10FA30007C180C0C6C044418242000006000040C9A
:10FA40002C6444606444447040180C50607C7C64B6
:10FA50004464442418646464183C18607C180000F2
:10FA6000000464606864486454180C78187C54641A
:10FA70006C6C5460306464643C640C30180C188006
:10FA800080841090C4F8806C04646440406C6C8086
:10FA9000C0A0888400000000808080808080FCB44A
:10FAA0001880442840844084808418308080282432
:10FAB00000440C40844444440000C00428241880BE
:10FAC00000000000000000000000C004C00440244A
:10FAD000A4B0BC4080808080E82CC8A488104084FA
:10FAE000E42400C4EC44F434E094C0048080208812
:10FAF000288020882088808020888020882CE8F03A
:10FB00000000000090909090101010108080808075
:10FB10007C8080801090B098408080440040646475
:10FB2000001800401C307800300C7C182800003091
:10FB300054181804400464186404282830400C1831
:10FB40007C4064606460606464180C78606468641D
:10FB5000607C780418643C7C3C1830600C18000011
:10FB6000002064606440306464180C50187C646445
:10FB70006C6C602430646464182C181818180C0C11
:10FB800080842088C4C444C420646430286C6C80A1
:10FB9000C0A08884000000008080808080807CEC91
:10FBA00018008044408440848080301880FC801895
:10FBB00000448040844444440000C004280024449D
:10FBC00000000000000000000000C004C004244049
:10FBD000BCD0A41084404084E82CC8A44C8480800D
:10FBE000482400C4EC44EC7CE094C004808020886D
:10FBF000288020882088808020888020882CE82801
:10FC00000000000090909090101010108080808074
:10FC1000FC8080801090808084C4A8440000643CF4
:10FC20000000003C44686C00181818181800286080
:10FC3000641830640C646430640C281818001800D0
:10FC40007C6464646460606464186C6C60646464A4
:10FC500060686C6418643C7C641860600018000084
:10FC6000006464646460302064180C781864646410
:10FC7000482460043C683C7C3C0830181818041880
:10FC800044882088C4C4808064646818186C6C80C0
:10FC9000C0A0888400000080808080808080FCB4C8
:10FCA000400080804084208880843018DC80284098
:10FCB00000446040844444280000C0046C0024C414
:10FCC00000000000000000000000C004C00418187C
:10FCD000BCB0808084402088E44CC4C44C848080C4
:10FCE000282400C4EC44F87CFCF4C00480002828DC
:10FCF000280028280000280028282820882CE83000
:10FD00000000000090909090101010108080808073
:10FD10007C4480441450808044EC442800004458C3
:10FD20000018003C18082C000C300000300028009F
:10FD3000242440240C242430242800300C003018C3
:10FD4000246444244440602464242864406464247B
:10FD5000602C64241824182464184048004800408B
:10FD6000002044242424300464246C6C246464241F
:10FD7000600C6044182C183C6404400C18300400DB
:10FD8000449040848080442820242C0000A8448093
:10FD9000C0A08884000080808080808040847C585F
:10FDA000240080288080208890A0600CDCFC44180F
:10FDB00000446040844444EC0000C0046C00240013
:10FDC00000000000000000000000C004C004104853
:10FDD000BCB0808080801090D094C0048C8040841F
:10FDE000284000C4C444F44CC004C0048000282847
:10FDF000280028280000280028282820882CE830FF
:10FE00000000000090909090101010108080808072
:10FE1000FC4480441450A8A84080440000006000C6
:10FE200000000000000000000000000000000000D2
:10FE300000000000000000000000000000000000C2
:10FE400000000000000000000000000000000000B2
:10FE500000000000000000000000000000000000A2
:10FE60000000000000000024000028000000000046
:10FE700060080000000000000024000000000000F6
:10FE800028A08080000000000000000000A844803E
:10FE9000C0A0888400808080808080804084FCECCA
:10FEA0001800444480801090A4A0C004DC806C3C06
:10FEB00000446000004400800080C004C4002400AE
:10FEC00000000000000000000000C004808000006E
:10FED000A4B08080844008A0C8A480808C800000EA
:10FEE000444000808000F47C4084C0040000282846
:10FEF000280028280000280028282824482CE8006A
:10FF00000000000090909090101010108080808071
:10FF10007C2880281450109080EC28000000C0003D
:10FF200000000000000000000000000000000000D1
:10FF300000000000000000000000000000000000C1
:10FF400000000000000000000000000000000000B1
:10FF500000000000000000000000000000000000A1
:10FF60000000000000000000000000000000000091
:10FF70000000000000000000000000000000000081
:10FF800028C0808000000000000000000000008009
:10FF9000C0A08884808080808080808020887C5879
:10FFA00000004480808008A004C0C0048CFCA858D5
:10FFB00000006000004400280080C004C40000006D
:10FFC00000000000000000000000C004000000006D
:10FFD0008080000084400000C8A400004824000085
:10FFE000000000000000C0040000C00480002828B9
:10FFF000280028280000280028282828282CE80085
:00000001FF
